:1000000032EF31F00000000000EF00F000000000CF
:0A0010000000000000000000F3D71C
:0E001C00ACB202D00000FCD73BC6ADFF120014
:0C002A0072B201D0FDD73BC673FF12007C
:10003600800E0601395D04E2400E3A5D01E201D010
:1000460060D0030E006E3AC604F0000E056E005036
:1000560004E00432049EFF0FFBD7070E006E000E6D
:10006600056E005005E0043604900536FF0FFAD7FA
:1000760039510426000E052200019F5321E0580E37
:100086000424026E010E0520036E070E06013A15C2
:10009600006E00C001F0010E006E015004E0003653
:1000A6000090FF0FFBD702C0E9FF03C0EAFFEE5046
:1000B600001202C0E1FF03C0E2FF00C0E6FF21D04C
:1000C6000601580E0424026E010E0520036E070E6B
:1000D6003A15006E00C001F0010E006E015004E0FA
:1000E60000360090FF0FFBD7001E02C0E9FF03C0D9
:1000F600EAFFEE50001602C0E1FF03C0E2FF00C0B7
:04010600E6FF1200FE
:10010A00C7B409D01F0EC514016E0150000A03E1DD
:0A011A00010E006E01D0006A120011
:10012400F250026EF29E0500FF6A0150FE6E00500E
:08013400FD6E02BEF28E120006
:10013C000B840BAEA9EF00F0010E036E026A016A8C
:0A014C00006A0A360232FF0E1200AC
:080156000AAE029E000E120029
:10015E00800E06013A19006E800E005C02E1000E60
:10016E00395D08E239510008006E3AC601F0000E02
:0E017E00015604D039C600F03AC601F0120056
:10018C000B820BAED0EF00F00368026801680068C8
:08019C000A360232FF0E1200C8
:0E01A400026A016A006A086A036A000E12000D
:1001B2000CB01BEF01F00CA2C1EF01F00E6A000EB1
:1001C200026432EF01F0F00E0214D8A4FDEF00F049
:1001D200023A01380F0B02260138F00B016E00388B
:1001E2000F0B01260038F00B006E08380F0B0026AB
:1001F2000838F00B086E0E84D89002BE16EF01F09C
:1002020008360036013602360E2A02BE16EF01F01B
:1002120008360036013602360E2A02BE16EF01F00B
:1002220008360036013602360E2A0E500364B7EF46
:1002320001F0035E0BBC08AEBCEF01F0D880800E6B
:1002420008640030000E002201220222D8A0BCEF76
:1002520001F0023201320032034AC1EF01F0BCEF79
:1002620001F001C002F000C001F008C000F0086A0D
:10027200000E0E86026469EF01F0F00E0214D8A49B
:1002820051EF01F0023A01380F0B02260138F00B50
:10029200016E00380F0B01260038F00B006E0E8441
:1002A200D89002BE16EF01F00036013602360E2A51
:1002B20002BE16EF01F00036013602360E2A02BEE9
:1002C20016EF01F00036013602360E2A16EF01F063
:1002D20001C002F000C001F0006A000E0E960E8806
:1002E200026496EF01F0F00E0214D8A481EF01F03F
:1002F200023A01380F0B02260138F00B016E0E8410
:10030200D89002BE16EF01F0013602360E2A02BE66
:1003120016EF01F0013602360E2A02BE16EF01F088
:10032200013602360E2A16EF01F001C002F0016A10
:10033200000E0E860264C6EF01F0F00E0214D8A47D
:10034200A5EF01F0023A0E84D89002BE16EF01F03A
:1003520002360E2A02BE16EF01F002360E2A02BE45
:1003620016EF01F002360E2A16EF01F0010E0C6EA6
:10037200E4DEC9EF01F0020E0C6EECDEC9EF01F013
:10038200040E0C6E02DFC9EF01F0080E0C6E09DFDD
:02039200120057
:1003940006012351275D396F245128593A6FDDDE58
:1003A40000C037F601C038F62151255D396F22515E
:1003B40026593A6FD2DE800E0118026E800E38196B
:1003C400025C02E13751005C010ED8B0000E026EEF
:1003D40002C031F6025218E021C629F622C62AF6D6
:1003E40023C621F624C622F629C623F62AC624F6F5
:1003F40025C62BF626C62CF627C625F628C626F6CD
:100404002BC627F62CC628F62251265D02E121517F
:10041400255D18E221C62DF622C62EF625C621F644
:1004240026C622F62DC625F62EC626F623C62FF698
:1004340024C630F627C623F628C624F62FC627F688
:1004440030C628F62151255D336F2351275D396F5E
:10045400245128593A6F81DE00C034F633C635F68C
:10046400000E366F3533359F000E366F2851245DEC
:1004740002E12751235D03E2010E326F02D0FF0E29
:10048400326F2251265D02E12151255D2CE3315367
:1004940006E023C639F621C63AF6CBDD05D021C6DF
:1004A40039F623C63AF6C5DD06013451355D016ED1
:1004B400000E3659026E01C035F602C036F6800EC3
:1004C4000218006E800E005C02E1000E015C08E27E
:1004D40032512327000E242333513527000E3623AF
:0804E400214B222BCED71200A0
:1004EC0015C023F616C024F617C025F618C026F63C
:1004FC000601216B226B2251120802E121518E0858
:10050C0008E3FDDD005201E004D00601214B222B53
:10051C00F2D70601120E225D02E18F0E215D03E37C
:10052C007B0E006E24D0C580C5A020D015501610AF
:10053C00171018101AE023512411251126110EE161
:10054C0040C1E1FF41C1E2FF050EE66E3EC100F085
:10055C003FC101F0E1DD010E006E09D0010E060174
:10056C00235F000E245B255B265BDED7006A12003E
:04057C00C584120020
:100580009E9621C6C9FF15C022F616C023F617C0D5
:1005900024F618C025F6C7A421D015501610171040
:1005A00018101BE0060122512311241125110EE120
:1005B00040C1E1FF41C1E2FF040EE66E3EC100F022
:1005C0003FC101F0AFDD010E006E3AD0010E060111
:1005D000225F000E235B245B255BDDD715C022F66E
:1005E00016C023F617C024F618C025F69EB621D0F3
:1005F00015501610171018101BE006012251231178
:10060000241125110EE140C1E1FF41C1E2FF040EBA
:10061000E66E3EC100F03FC101F084DD010E006EC8
:100620000FD0010E0601225F000E235B245B255BC9
:10063000DDD7C5BC02D0006A03D0C584020E006EAF
:020640001200A6
:080642000B6A0B86FF0E12008B
:10064A000B6A0A6A096A00500402F4CF09F0F3CF70
:10065A0008F001500502F4CF0BF0F3CF0AF0005076
:10066A000502F3500926F4500A22E86A0B220150C7
:10067A000402F3500926F4500A22E86A0B2208C041
:10068A0000F009C001F00AC002F00BC003F012002A
:10069A000450085E0550D8A0053C095E0650D8A053
:1006AA00063C0A5E0750D8A0073C0B5E0336070ECD
:1006BA000C6E0334083609360A360B36045003A08A
:1006CA000ED0085E0550D8A0053C095E0650D8A099
:1006DA00063C0A5E0750D8A0073C0B5E0DD00826E0
:1006EA000550D8B0053C09260650D8B0063C0A2663
:1006FA000750D8B0073C0B2603360C2EDAD7023443
:10070A00083609360A360B36045003A00ED0085EA6
:10071A000550D8A0053C095E0650D8A0063C0A5EE2
:10072A000750D8A0073C0B5E0DD008260550D8B05C
:10073A00053C09260650D8B0063C0A260750D8B010
:10074A00073C0B260236070E0C6E023408360936B1
:10075A000A360B36045002A00ED0085E0550D8A007
:10076A00053C095E0650D8A0063C0A5E0750D8A090
:10077A00073C0B5E0DD008260550D8B0053C09266B
:10078A000650D8B0063C0A260750D8B0073C0B26BC
:10079A0002360C2EDAD70134083609360A360B36F9
:1007AA00045002A00ED0085E0550D8A0053C095E90
:1007BA000650D8A0063C0A5E0750D8A0073C0B5E3C
:1007CA000DD008260550D8B0053C09260650D8B0E9
:1007DA00063C0A260750D8B0073C0B260136070EFE
:1007EA000C6E0134083609360A360B36045001A05D
:1007FA000ED0085E0550D8A0053C095E0650D8A068
:10080A00063C0A5E0750D8A0073C0B5E0DD00826AE
:10081A000550D8B0053C09260650D8B0063C0A2631
:10082A000750D8B0073C0B2601360C2EDAD7003415
:10083A00083609360A360B36045001A00ED0085E77
:10084A000550D8A0053C095E0650D8A0063C0A5EB1
:10085A000750D8A0073C0B5E0DD008260550D8B02B
:10086A00053C09260650D8B0063C0A260750D8B0DF
:10087A00073C0B260036070E0C6E00340836093684
:10088A000A360B36045000A00ED0085E0550D8A0D8
:10089A00053C095E0650D8A0063C0A5E0750D8A05F
:1008AA00073C0B5E0DD008260550D8B0053C09263A
:1008BA000650D8B0063C0A260750D8B0073C0B268B
:1008CA0000360C2EDAD700B00ED004500826055098
:1008DA00D8B0053C09260650D8B0063C0A2607506F
:0808EA00D8B0073C0B261200F8
:1008F200025006180E6E086A096A0B6A03500764F2
:100902006CEF05F006500A6E068E028E03500B6ED7
:100912000750036E000E0B64BCEF04F00B50075E31
:10092200D8B45DEF05F0070E07642BEF05F0075E04
:1009320000C008F001C000F002C001F0026A074ED8
:100942005DEF05F0076400EF05F0075E00C008F0F8
:1009520001C000F0016A074E5DEF05F00764DEEFAB
:1009620004F0075E00C008F0006A074E5DEF05F074
:100972000764C5EF04F00AC002F005C001F004C02C
:1009820000F0086A89EF06F0030E0764D0EF04F066
:10099200075E08380F0B086E074E5DEF05F0D89022
:1009A2000832074E5DEF05F0D8900832074E5DEF32
:1009B20005F0D89008325DEF05F0030E0764EFEF03
:1009C20004F0075E08380F0B086E0038F00B08269B
:1009D20000380F0B006E074E5DEF05F0D890003225
:1009E2000832074E5DEF05F0D89000320832074E0C
:1009F2005DEF05F0D890003208325DEF05F0030E8E
:100A0200076417EF05F0075E08380F0B086E003811
:100A1200F00B082600380F0B006E0138F00B002691
:100A220001380F0B016E074E5DEF05F0D8900132D1
:100A320000320832074E5DEF05F0D89001320032E5
:100A42000832074E5DEF05F0D890013200320832CD
:100A52005DEF05F0030E076448EF05F0075E083806
:100A62000F0B086E0038F00B082600380F0B006ED3
:100A72000138F00B002601380F0B016E0238F00B23
:100A8200012602380F0B026E074E5DEF05F0D8907B
:100A92000232013200320832074E5DEF05F0D89083
:100AA2000232013200320832074E5DEF05F0D89073
:100AB2000232013200320832096A000E0EAE51EFE4
:100AC20006F0081E001E011E021E082A0022012234
:100AD200022251EF06F00750D8A472EF05F089EF19
:100AE20006F0096A02C00AF0028E068E0750035C05
:100AF200076ED8B444EF06F0070E076412EF06F053
:100B0200075E0450096E0550046E0650056E066AB3
:100B1200074E44EF06F0070E0764E7EF05F0075EA5
:100B22000450096E0550046E056A074E44EF06F044
:100B3200070E0764C5EF05F0075E0450096E046AEC
:100B4200074E44EF06F0070E0764ACEF05F00AC04B
:100B520002F089EF06F0030E0764B7EF05F0075EB7
:100B620009380F0B096E074E44EF06F0D890093290
:100B7200074E44EF06F0D8900932074E44EF06F0D4
:100B8200D890093244EF06F0030E0764D6EF05F061
:100B9200075E09380F0B096E0438F00B092604387A
:100BA2000F0B046E074E44EF06F0D8900432093260
:100BB200074E44EF06F0D89004320932074E44EF54
:100BC20006F0D8900432093244EF06F0030E0764AF
:100BD200FEEF05F0075E09380F0B096E0438F00BC3
:100BE200092604380F0B046E0538F00B042605386D
:100BF2000F0B056E074E44EF06F0D8900532043213
:100C02000932074E44EF06F0D89005320432093219
:100C1200074E44EF06F0D89005320432093244EF11
:100C220006F0030E07642FEF06F0075E09380F0B7C
:100C3200096E0438F00B092604380F0B046E0538D0
:100C4200F00B042605380F0B056E0638F00B05264F
:100C520006380F0B066E074E44EF06F0D8900632A8
:100C6200053204320932074E44EF06F0D8900632BC
:100C7200053204320932074E44EF06F0D8900632AC
:100C8200053204320932086A000E0EAE51EF06F048
:100C9200091E041E051E061E092A0422052206221A
:100CA2000950082604500022055001220650022253
:100CB2000EBE68EF06F0D8A077EF06F002320132DE
:100CC20000320832033E77EF06F083EF06F0D8B029
:100CD2007DEF06F0000E081E001E011E021E082AED
:100CE2000022012202220A7E7DEF06F0010E0C6E26
:100CF200D9EC00F08BEF06F0020E0C6ED9EC00F08E
:100D02008BEF06F0040E0C6EC6EC00F08BEF06F0D3
:060D1200000E0C6E120041
:100D18000B800BAE98EF06F0026A0AAEFF0E026E69
:0C0D2800016E006E0A360232FF0E12004F
:100D34001EC621F6000E0601226F1FC623F6000E02
:100D4400246F1EC625F6000E266F20511F25276F1F
:100D5400286B000E2823010E275F000E285BCAECC7
:040D640001F0120088
:100D68000B1E0A1E091E081E082AD8B4092AD8B460
:080D78000A2AD8B40B2A12006C
:100D80000134083609360450085E0550D8A0053CE9
:100D9000095E003601360F0E0C6E01340836093636
:100DA000045000A006D0085E0550D8A0053C095E9E
:100DB00005D008260550D8B0053C09260036013676
:100DC0000C2EEBD700B006D0045008260550D8B042
:080DD000053C09260000120099
:100DD800086A080E0C6E003408360450085ED8B055
:0E0DE80002D00826D89000360C2EF5D7120047
:100DF60076EC02F0780E0601216FC0EC02F085EC6D
:100E060000F00050000A01E1FAD7800E0601216FBA
:100E1600C0EC02F085EC00F00050000A01E1FAD7C0
:100E26001EC621F6C0EC02F085EC00F00050000A68
:0A0E360001E1FAD7BEEC02F0120051
:100E4000086A096A000E07620364A5EF07F0025002
:100E500006180A6E075003267E0ED8A036EF07F05C
:100E6000035ED8B0AAEF07F03AEF07F0035ED8A010
:100E7000AFEF07F0028E068E02C00EF001C00BF03D
:100E800000C00DF000500402F4CF0CF00150050238
:100E9000F4CF00F0F3CF08F00402F3500C26F45026
:100EA0000822000E00220D500502F3500C26F450CB
:100EB0000822000E002202500402F3500826F450CB
:100EC000002202500502016A000E0122F3500026A2
:100ED000F45001220D500602F3500826F45000226F
:100EE000026A000E012202220B500602F350002675
:100EF000F4500122000E02220E500602F350012689
:100F0000F450022202BE8DEF07F00836003601369B
:100F100002360306D8B4AFEF07F0A0EF07F0D88091
:100F2000800E08640030000E002201220222D8A0A8
:100F3000A0EF07F0023201320032034AAAEF07F0B5
:100F40000AAE029E000EB2EF07F0010ED2EC00F0E6
:100F5000B2EF07F0020EC6EC00F0B2EF07F0040E9D
:060F60009EEC00F01200FF
:100F66000D6A086A0050D8B4000C04180A6E0ABE4E
:100F76000D1E0B6A04AE02D0041E042A00AE02D077
:100F8600001E002A005004100A6E0ABE1FD004502C
:100F9600085E003600340836045008260036060E71
:100FA6000C6E00340836045000B0085E00A0082617
:100FB60000360C2EF6D700A008260BB015D00DAEC5
:100FC600000C001E002A081E082A000C04AE09D0D8
:100FD60000BE04D00050086E006AF1D7006A002AED
:100FE600000C001E0B2AD3D7082A0450085CD8A48C
:0E0FF600E6D7086A002A00AEE2D7FF0C120010
:1010040006010F510108146F10C615F6000E15578E
:10101400010E1A6F000E1B6FFE0E006EFF0E016EA6
:101024000FC604F010C605F025EC03F000C016F658
:1010340001C017F61C6B1D6B0FC618F610C619F607
:10104400800E1D19006E800E1919005C02E1185102
:101054001C5D68E2800E1519006E800E005C02E1D2
:10106400000E145D12E3010E185F000E195B020EF0
:101074001625006E000E1721016E00C016F601C081
:1010840017F600501427015015231C4B1D2B020E7C
:101094001A25006E000E1B21016E00C01AF601C055
:1010A4001BF6005014270150152311A11CD01C510C
:1010B4000B251E6F18510D5D1F6F18C620F62037C3
:1010C4002091202B1251202733DE18510B251E6F3F
:1010D4001C510D5D1F6F1CC620F620372091202B5C
:1010E4001251202725DE11A31CD01C510B5D1E6F4D
:1010F40018510D5D1F6F18C620F620372091202B44
:101104001251202715DE18510B5D1E6F1C510D5D09
:101114001F6F1CC620F620372091202B1251202748
:0611240007DE8ED7120069
:10112A006E0E06010B5DD8A0C3D0640E046E0BC60A
:10113A0000F04DDE120E0024056E066A000E06222D
:10114A0005C000F006C001F0000E06BEFF0E026EDA
:10115A00036E0036009001360236033600360090E0
:10116A00013602360336CF0E0024F66E870E0120B2
:10117A00F76E000E0220F86E0900F5CF00F00900A4
:10118A00F5CF01F00900F5CF02F00900F5CF03F021
:10119A00000E046E000E056E000E066E7E0E076EC1
:1011AA004ADE00C00CF601C00DF602C00EF603C0FE
:1011BA000FF6640E046E0BC600F009DE08C000F0DC
:1011CA000A0E046E04DE090E0024056E066A000E7D
:1011DA00062205C000F006C001F0000E06BEFF0E92
:1011EA00026E036E00360090013602360336003670
:1011FA000090013602360336CF0E0024F66E870EB3
:10120A000120F76E000E0220F86E0900F5CF00F0FB
:10121A000900F5CF01F00900F5CF02F00900F5CF7A
:10122A0003F00CC604F00DC605F00EC606F00FC694
:10123A0007F001DE00C00CF601C00DF602C00EF682
:10124A0003C00FF60A0E046E0BC600F0C0DD08C01C
:10125A0000F000C001F0000E026E036E046E01364B
:10126A0001900236033604360136019002360336FF
:10127A000436CF0E0124F66E870E0220F76E000E9A
:10128A000320F86E0900F5CF00F00900F5CF01F050
:10129A000900F5CF02F00900F5CF03F00CC604F0FF
:1012AA000DC605F00EC606F00FC607F0C4DDACD0B9
:1012BA000B510A08D8B07AD00A0E046E0BC600F099
:1012CA0086DD090E0024056E066A000E062205C098
:1012DA0000F006C001F0000E06BEFF0E026E036E9D
:1012EA000036009001360236033600360090013689
:1012FA0002360336CF0E0024F66E870E0120F76EF3
:10130A00000E0220F86E0900F5CF00F00900F5CFB3
:10131A0001F00900F5CF02F00900F5CF03F0000E45
:10132A00046E000E056E000E066E7E0E076E83DDDD
:10133A0000C00CF601C00DF602C00EF603C00FF68F
:10134A000A0E046E0BC600F042DD08C000F000C0B1
:10135A0001F0000E026E036E046E01360190023631
:10136A000336043601360190023603360436CF0EB0
:10137A000124F66E870E0220F76E000E0320F86E27
:10138A000900F5CF00F00900F5CF01F00900F5CF0B
:10139A0002F00900F5CF03F00CC604F00DC605F003
:1013AA000EC606F00FC607F046DD2ED00BC600F0BB
:1013BA00000E016E026E036E003600900136023690
:1013CA00033600360090013602360336CF0E00246B
:1013DA00F66E870E0120F76E000E0220F86E0900E5
:1013EA00F5CF00F00900F5CF01F00900F5CF02F0C2
:1013FA000900F5CF03F0000E046E000E056E000E14
:0A140A00066E7E0E076E17DD12005D
:10141400520E0B6E2B0E0C6E000E0D6E0D2EFED7A3
:0C1424000C2EFCD70B2EFAD70000120093
:101430000450000A12E10550000A0FE10650000AAC
:101440000CE10750000A09E1FF0E006EFF0E016E6D
:101450007F0E026EFF0E036EA8D0086A096A07505D
:10146000D8B4C3EF0AF00350D8B4C8EF0AF0025062
:1014700006180A6E028E068E0E6A02C008F001C0BF
:101480000CF000C00DF004500D5E0550D8A0053CD6
:101490000C5E0650D8A0063C085E086A0C6A0D6A0D
:1014A000D8A05AEF0AF0D890023201320032083246
:1014B000010E0E6E0750035ED8A067EF0AF07E0E95
:1014C0000E240326D8B0CDEF0AF06DEF0AF07E0EA1
:1014D0000E240326D8A0D2EF0AF0180E0B6E0D369C
:1014E0000C3608360036013602360E360450005EE1
:1014F0000550D8A0053C015E0650D8A0063C025E0F
:1015000006340E120EA088EF0AF00D8093EF0AF059
:10151000045000260550D8B0053C01260650D8B02E
:10152000062802260D900B2E6FEF0AF0B9EF0AF095
:10153000D8900036013602360E360450005E055053
:10154000D8A0053C015E0650D8A0063C025E0634D9
:101550000E10010B0D26D8B00C2AD8B4082AD8A436
:10156000B9EF0AF008320C320D32032AD8B4CDEFAD
:101570000AF00AAE089E0850026E0C50016E0D5023
:10158000006ED5EF0AF0010E21EC03F0D5EF0AF062
:10159000020ED2EC00F0D5EF0AF0040EC6EC00F01B
:0C15A000D5EF0AF0080E9EEC00F01200DF
:1015AC0006010B51390806E3300E0B5D03E3010E07
:0815BC00006E01D0006A12006C
:1015C400220E0C6E086A096A0A6A0B6A0C06D8B401
:1015D4001FD0D8900B320A32093208320332023259
:1015E40001320032D8A0F2D70C06D8B409D0045086
:1015F40008260550092206500A2207500B22EAD772
:10160400045008260550092206500A2207500B22CE
:021614001200C2
:101616000A6A0350D8A40A800750D8A40A820A503E
:10162600D8B46EEF0BF0030AD8B427EF0BF00AB06C
:1016360022EF0BF006AE6CEF0BF06AEF0BF002AE8A
:101646006AEF0BF06CEF0BF00250800B0A6E029EF5
:101656000650800B069E0A18D8B438EF0BF00A50D5
:10166600D8B46AEF0BF06CEF0BF00750035CD8B4FC
:1016760042EF0BF0D8A05EEF0BF064EF0BF00650D4
:10168600025CD8B44CEF0BF0D8A05EEF0BF064EF21
:101696000BF00550015CD8B456EF0BF0D8A05EEF06
:1016A6000BF064EF0BF00450005CD8B46EEF0BF057
:1016B600D8B064EF0BF00A52D8B46CEF0BF06AEFB7
:1016C6000BF00A52D8B46AEF0BF06CEF0BF0D8802F
:0E16D6001200D8901200D880D88412001200A2
:1016E4000B6A0C6A086A0350D8B4F6EF0BF002C018
:1016F4000AF0028E9E0E035E03AEE6EF0BF0036C5F
:10170400080E035CD8A0B3EF0BF0036E083600C0DC
:1017140008F001C000F002C001F0026A080E035C88
:10172400D8A0B3EF0BF0036E083600C008F001C078
:1017340000F0016A080E035CD8A0B3EF0BF0036E4F
:10174400083600C008F0006A080E035CD8A0B3EFA6
:101754000BF0036E0836086A0350D8A4D890BFEF84
:101764000BF00350D8B4BFEF0BF0D8900232013223
:1017740000320832032EB7EF0BF00BBC08A0D0EFF9
:101784000BF0D8A0D0EF0BF0082AD8B4002AD8B4B4
:10179400012AD8B4022A02BEFAEF0BF00AAEF6EF21
:1017A4000BF0021E011E001E081E082AD8B4002ACF
:1017B400D8B4012AD8B4022AF6EF0BF0026A016AFF
:1017C400006A086AF6EF0BF00B800BAE01EF0CF029
:1017D400026A0AAE01EF0CF0026E016E006E086E32
:1017E4000A36023201EF0CF00C6A000E02EF0CF024
:1017F400010E0C6E000E8CEC06F002EF0CF0FF0EE6
:101804000250036E0150026E0050016E0850006ECB
:021814001200C0
:1018160076EC02F0780E0601216FC0EC02F085EC42
:1018260000F00050000A01E1FAD70601216BC0EC76
:1018360002F085EC00F00050000A01E1FAD70BC671
:1018460021F6C0EC02F085EC00F00050000A01E140
:10185600FAD7BEEC02F085EC00F00050000A01E178
:04186600FAD712009B
:10186A000B6A0A6A096A086A0E6A0334083604505F
:10187A00085E0550D8A0053C095E0650D8A0063C73
:10188A000A5E0750D8A0073C0B5EE86AD8A0010E92
:10189A000E5E0336070E0C6E0334083609360A3616
:1018AA000B360E36045003A012D0085E0550D8A09D
:1018BA00053C095E0650D8A0063C0A5E0750D8A02F
:1018CA00073C0B5EE86AD8A0010E0E5E11D008260E
:1018DA000550D8B0053C09260650D8B0063C0A2661
:1018EA000750D8B0073C0B26E86AD8B0010E0E267E
:1018FA0003360C2ED1D70234083609360A360B368F
:10190A000E36045003A012D0085E0550D8A0053C3C
:10191A00095E0650D8A0063C0A5E0750D8A0073CCC
:10192A000B5EE86AD8A0010E0E5E11D0082605509B
:10193A00D8B0053C09260650D8B0063C0A260750FE
:10194A00D8B0073C0B26E86AD8B0010E0E2602363C
:10195A00070E0C6E0234083609360A360B360E3676
:10196A00045002A012D0085E0550D8A0053C095EBA
:10197A000650D8A0063C0A5E0750D8A0073C0B5E6A
:10198A00E86AD8A0010E0E5E11D008260550D8B01C
:10199A00053C09260650D8B0063C0A260750D8B09E
:1019AA00073C0B26E86AD8B0010E0E2602360C2E2A
:1019BA00D1D70134083609360A360B360E360450AA
:1019CA0002A012D0085E0550D8A0053C095E065058
:1019DA00D8A0063C0A5E0750D8A0073C0B5EE86A0E
:1019EA00D8A0010E0E5E11D008260550D8B0053CCD
:1019FA0009260650D8B0063C0A260750D8B0073C3C
:101A0A000B26E86AD8B0010E0E260136070E0C6EB8
:101A1A000134083609360A360B360E36045001A050
:101A2A0012D0085E0550D8A0053C095E0650D8A021
:101A3A00063C0A5E0750D8A0073C0B5EE86AD8A0AD
:101A4A00010E0E5E11D008260550D8B0053C0926B5
:101A5A000650D8B0063C0A260750D8B0073C0B26D9
:101A6A00E86AD8B0010E0E2601360C2ED1D7003402
:101A7A00083609360A360B360E36045001A012D043
:101A8A00085E0550D8A0053C095E0650D8A0063C61
:101A9A000A5E0750D8A0073C0B5EE86AD8A0010E80
:101AAA000E5E11D008260550D8B0053C092606500E
:101ABA00D8B0063C0A260750D8B0073C0B26E86A7D
:101ACA00D8B0010E0E260036070E0C6E003408360A
:101ADA0009360A360B360E36045000A012D0085EBC
:101AEA000550D8A0053C095E0650D8A0063C0A5EFF
:101AFA000750D8A0073C0B5EE86AD8A0010E0E5E1C
:101B0A0011D008260550D8B0053C09260650D8B091
:101B1A00063C0A260750D8B0073C0B26E86AD8B01C
:101B2A00010E0E2600360C2ED1D700B00ED004506E
:101B3A0008260550D8B0053C09260650D8B0063C00
:0C1B4A000A260750D8B0073C0B261200FA
:101B56000450000A08E10550000A05E1FF0E006E78
:101B66007F0E016E58D00D6A096A086A015000108E
:101B7600D8B4000C015005180A6E0ABE0D1E0B6A79
:101B860005AE05D0041E051E042AD8B4052A01AEEA
:101B960005D0001E011E002AD8B4012A01500510E6
:101BA6000A6E0ABE10D0C0EC06F00BB020D00DAE07
:101BB600000C001E011E002AD8B4012A081E091EA8
:101BC600082AD8B4092A000C05AE0DD001BE07D0EC
:101BD6000150096E0050086E016A006AE8D7016A72
:101BE600006A002A000C011E001E0B2ADDD7082AF7
:101BF600D8B4092A0450085CD8A4D9D70550095C82
:101C0600D8A4D5D7096A086A002AD8B4012A01AE31
:081C1600CED70000FF0C120004
:101C1E0003500718D8A423EF0EF002500618D8A4CC
:101C2E0023EF0EF001500518D8A423EF0EF000504C
:0E1C3E000418D8B4D8841200D89412001200F2
:101C4C00800E06010B19006E800E000A005CD8B0E5
:101C5C006DD10B510008016E01C00BF6800E0118FE
:101C6C00006E800E6E0A005CD8A0C0D0640E046EAC
:101C7C000BC600F0B3EC07F0120E0024056E000E3C
:101C8C0000BEFF0E066E000E062205C000F006C058
:101C9C0001F0000E06BEFF0E026E036E00360090C1
:101CAC000136023603360036009001360236033612
:101CBC00CF0E0024F66E870E0120F76E000E022068
:101CCC00F86E0900F5CF0CF60900F5CF0DF60900FA
:101CDC00F5CF0EF60900F5CF0FF6640E046E0BC6A9
:101CEC0000F0B3EC07F008C000F00A0E046EB3EC81
:101CFC0007F0090E0024056E000E00BEFF0E066EE6
:101D0C00000E062205C000F006C001F0000E06BE53
:101D1C00FF0E026E036E003600900136023603365B
:101D2C0000360090013602360336CF0E0024F66ED4
:101D3C00870E0120F76E000E0220F86E0900F5CF19
:101D4C0000F00900F5CF01F00900F5CF02F0090011
:101D5C00F5CF03F00CC604F00DC605F00EC606F068
:101D6C000FC607F020EC07F000C00CF601C00DF612
:101D7C0002C00EF603C00FF60A0E046E0BC600F07E
:101D8C00B3EC07F008C000F000C001F0000E00BE7C
:101D9C00FF0E026E036E046E01360190023603369E
:101DAC00043601360190023603360436CF0E012478
:101DBC00F66E870E0220F76E000E0320F86E0900F7
:101DCC00F5CF00F00900F5CF01F00900F5CF02F0D6
:101DDC000900F5CF03F00CC604F00DC605F00EC6D5
:101DEC0006F00FC607F020EC07F007D2800E0A0AA7
:101DFC00006E800E0B19005C71E20A0E046E0BC6AD
:101E0C0000F0B3EC07F0090E0024056E000E00BEC6
:101E1C00FF0E066E000E062205C000F006C001F093
:101E2C00000E06BEFF0E026E036E003600900136E9
:101E3C000236033600360090013602360336CF0EDA
:101E4C000024F66E870E0120F76E000E0220F86E4D
:101E5C000900F5CF0CF60900F5CF0DF60900F5CF0A
:101E6C000EF60900F5CF0FF60A0E046E0BC600F045
:101E7C00B3EC07F008C000F000C001F0000E00BE8B
:101E8C00FF0E026E036E046E0136019002360336AD
:101E9C00043601360190023603360436CF0E012487
:101EAC00F66E870E0220F76E000E0320F86E090006
:101EBC00F5CF00F00900F5CF01F00900F5CF02F0E5
:101ECC000900F5CF03F00CC604F00DC605F00EC6E4
:101EDC0006F00FC607F020EC07F08FD10BC600F010
:101EEC00000E0BBFFF0E016E026E036E00360090EB
:101EFC0001360236033600360090013602360336C0
:101F0C00CF0E0024F66E870E0120F76E000E022015
:101F1C00F86E0900F5CF00F00900F5CF01F00900CB
:101F2C00F5CF02F00900F5CF03F067D1800E0B1945
:101F3C00006E800E6E0A005CD8A0C0D0640E046ED9
:101F4C000BC600F0B3EC07F0120E0024056E000E69
:101F5C0000BEFF0E066E000E062205C000F006C085
:101F6C0001F0000E06BEFF0E026E036E00360090EE
:101F7C00013602360336003600900136023603363F
:101F8C009B0E0024F66E870E0120F76E000E0220C9
:101F9C00F86E0900F5CF0CF60900F5CF0DF6090027
:101FAC00F5CF0EF60900F5CF0FF6640E046E0BC6D6
:101FBC0000F0B3EC07F008C000F00A0E046EB3ECAE
:101FCC0007F0090E0024056E000E00BEFF0E066E13
:101FDC00000E062205C000F006C001F0000E06BE81
:101FEC00FF0E026E036E0036009001360236033689
:101FFC00003600900136023603369B0E0024F66E36
:10200C00870E0120F76E000E0220F86E0900F5CF46
:10201C0000F00900F5CF01F00900F5CF02F009003E
:10202C00F5CF03F00CC604F00DC605F00EC606F095
:10203C000FC607F020EC07F000C00CF601C00DF63F
:10204C0002C00EF603C00FF60A0E046E0BC600F0AB
:10205C00B3EC07F008C000F000C001F0000E00BEA9
:10206C00FF0E026E036E046E0136019002360336CB
:10207C000436013601900236033604369B0E0124D9
:10208C00F66E870E0220F76E000E0320F86E090024
:10209C00F5CF00F00900F5CF01F00900F5CF02F003
:1020AC000900F5CF03F00CC604F00DC605F00EC602
:1020BC0006F00FC607F020EC07F09FD0800E0A0A3E
:1020CC00006E800E0B19005C71E20A0E046E0BC6DA
:1020DC0000F0B3EC07F0090E0024056E000E00BEF4
:1020EC00FF0E066E000E062205C000F006C001F0C1
:1020FC00000E06BEFF0E026E036E00360090013617
:10210C0002360336003600900136023603369B0E3B
:10211C000024F66E870E0120F76E000E0220F86E7A
:10212C000900F5CF0CF60900F5CF0DF60900F5CF37
:10213C000EF60900F5CF0FF60A0E046E0BC600F072
:10214C00B3EC07F008C000F000C001F0000E00BEB8
:10215C00FF0E026E036E046E0136019002360336DA
:10216C000436013601900236033604369B0E0124E8
:10217C00F66E870E0220F76E000E0320F86E090033
:10218C00F5CF00F00900F5CF01F00900F5CF02F012
:10219C000900F5CF03F00CC604F00DC605F00EC611
:1021AC0006F00FC607F020EC07F027D00BC600F0A6
:1021BC00000E0BBFFF0E016E026E036E0036009018
:1021CC0001360236033600360090013602360336ED
:1021DC009B0E0024F66E870E0120F76E000E022077
:1021EC00F86E0900F5CF00F00900F5CF01F00900F9
:0C21FC00F5CF02F00900F5CF03F012004F
:08220800067E79EC04F01200DF
:102210000050086E0150006E0250016E0350026EB5
:10222000036A0B6A0C6A9E0E036E0A6A020E0C6E3B
:06223000D9EC00F01200E1
:102236000450000A12E10550000A0FE10650000A98
:102246000CE10750000A09E1FF0E006EFF0E016E59
:10225600FF0E026E7F0E036E99D00C6A07BE0C2A23
:102266000D6A0B6A0A6A096A086A035002100110AD
:102276000010D8B485D0035007180E6E0EBE0D1E82
:1022860007AE0BD0041E051E061E071E042AD8B470
:10229600052AD8B4062AD8B4072A03AE0BD0001EE6
:1022A600011E021E031E002AD8B4012AD8B4022A2F
:1022B600D8B4032A035007100E6E0EBE1DD04DEC87
:1022C60003F00CBE36D00DAE5BD0001E011E021E02
:1022D600031E002AD8B4012AD8B4022AD8B4032A85
:1022E600081E091E0A1E0B1E082AD8B4092AD8B4CD
:1022F6000A2AD8B40B2A44D007AE15D003BE0DD097
:1023060003500B6E02500A6E0150096E0050086EA3
:10231600036A026A016A006AD6D7036A026A016A18
:10232600006A002A000C031E021E011E001E0C8EEF
:10233600C6D7082AD8B4092AD8B40A2AD8B40B2A88
:102346000450085CD8A4BFD70550095CD8A4BBD7F5
:1023560006500A5CD8A4B7D707500B5CD8A4B3D7ED
:102366000B6A0A6A096A086A002AD8B4012AD8B42C
:10237600022AD8B4032A03AEA6D70E6A0E88FF0C2B
:0E2386000E6A0CA002D0B4EC06F0000F12009C
:1023940006010F510108126F10C613F6000E1357F1
:1023A400010E186F000E196FFE0E006EFF0E016E07
:1023B4000FC604F010C605F025EC03F000C014F6B7
:1023C40001C015F61A6B1B6B0FC616F610C617F66E
:1023D4000601800E1B19006E800E1719005C02E1C5
:1023E40016511A5DD8B07BD0800E1319006E800E82
:1023F400005C02E1000E125D12E3010E165F000E96
:10240400175B020E1425006E000E1521016E00C02C
:1024140014F601C015F600501227015013231A4B6D
:102424001B2B020E1825006E000E1921016E00C030
:1024340018F601C019F6005012270150132311A5F4
:1024440011D01A510B25396F16510D253A6F1BEC1B
:1024540000F0060116510B25396F1A510D253A6FFC
:102464001BEC00F0060111A311D01A510B25396F92
:1024740016510D5D3A6F1BEC00F0060116510B2549
:10248400396F1A510D5D3A6F1BEC00F0060111A76C
:1024940011D016510B5D396F1A510D253A6F1BEC93
:1024A40000F006011A510B5D396F16510D253A6F74
:1024B4001BEC00F0060111A111D016510B5D396F10
:1024C4001A510D5D3A6F1BEC00F006011A510B5DB9
:1024D400396F16510D5D3A6F1BEC00F079D712007D
:1024E4000B6A0C6A0A6A086A0350D8B4FAEF12F04D
:1024F400028E9E0E035E03BE85EF12F0D8B485EF04
:1025040012F0EAEF12F0036C080E035CD8A0B7EFE8
:1025140012F0036E083600C008F001C000F002C0DB
:1025240001F0026A080E035CD8A0B7EF12F0036E44
:10253400083600C008F001C000F0016A080E035C10
:10254400D8A0B7EF12F0036E083600C008F0006A96
:10255400080E035CD8A0B7EF12F0036E0836086AC1
:102564000350D8A4D890C3EF12F00350D8B4C3EFEB
:1025740012F0D8900232013200320832032EBBEF3F
:1025840012F00BBC08A0D4EF12F0D8A0D4EF12F0D4
:10259400082AD8B4002AD8B4012AD8B4022A02BE20
:1025A400FEEF12F00AAEFAEF12F0021E011E001E38
:1025B400081E082AD8B4002AD8B4012AD8B4022A9A
:1025C400FAEF12F0026A016A006A086AFAEF12F07E
:1025D4000B800BAE04EF13F0026A0AAE04EF13F0A3
:1025E400026E016E006E086E0A36023204EF13F0BA
:1025F400000E0C6A05EF13F0010E0C6E8CEC06F065
:1026040005EF13F0FF0E0250036E0150026E0050EE
:08261400016E0850006E120077
:10261C000BC621F6000E0601226F0CC623F6000E27
:10262C00246F0D510B25256F266B000E2623010EF2
:10263C00255F000E265B0CC627F6000E286FCAEC31
:04264C0001F0120087
:102650000BC60FF6000E0601106F0D510B25016E13
:10266000026A000E02220250105D02E101500F5D6D
:102670000BE20FC61EF60CC61FF60EC620F69AEC2D
:0A26800006F00F4B102BE9D71200F3
:10268A0006010C51B00F1E6FFBEC06F00F0E06018F
:10269A000B151E6FFBEC06F0F00E06010B151E6FF4
:1026AA001E331E9F1E331E9F1E331E9F1E331E9FE8
:0826BA001E89FBEC06F0120082
:1026C2000BC602F00CC603F002C000F003C001F01A
:1026D200024A032A00C0E9FF01C0EAFFEE5201E00C
:1026E200F3D706010B51025C006E0C510358016EC8
:0A26F200010E005E000E015A1200F6
:1026FC0076EC02F0780E0601216FC0EC02F085EC4E
:10270C0000F00050000A01E1FAD7400E0601216FDB
:10271C00C0EC02F085EC00F00050000A01E1FAD7A1
:10272C000BC621F6C0EC02F085EC00F00050000A5C
:0A273C0001E1FAD7BEEC02F0120032
:10274600D1C504F0D2C505F004C0E9FF05C0EAFF13
:10275600EE5203E0044A052AF7D704C002F005C08A
:1027660003F0044A052AD3C500F0D4C501F00501DB
:10277600D34BD42B00C0E9FF01C0EAFF02C0E1FF42
:1027860003C0E2FFEECFE6FF02C0E9FF03C0EAFFA7
:10279600EE5201E0E2D7D1C500F0D2C501F0120039
:1027A6000501D46BD1C5E9FFD2C5EAFFEECFD3F55B
:1027B600D351000A0FE0D3C53BF60EEC00F005013D
:1027C600D42BD451D125E96E000ED221EA6EEECF7C
:0627D600D3F5EED712005E
:1027DC00D1C5F6FFD2C5F7FFD3C5F8FF0900F5CF79
:1027EC0000F0005212E0D1C5F6FFD2C5F7FFD3C5F9
:1027FC00F8FF0900F5CF3BF60EEC00F0010E0501D9
:0C280C00D127000ED223D323E3D7120003
:102818000501F16BF26BE56BE66BD3C500F0D4C52F
:1028280001F0D5C502F0010ED327000ED423D5231D
:1028380000C0F6FF01C0F7FF02C0F8FF0900F5CF9E
:1028480000F000C0E2F50052D8B42DEF24F0E251B8
:10285800250A0BE0D1C5E1FFD2C5E2FFE2C5E6FFDC
:10286800D14BD22BF14BF22BD8D7E36BE46BE56B52
:10287800E66B23D0E587010ED327000ED423D5239A
:1028880059D0E581010ED327000ED423D52352D089
:10289800E583010ED327000ED423D5234BD0E6873A
:1028A800010ED327000ED423D52344D0E585010E8D
:1028B800D327000ED423D5233DD0D3C5F6FFD4C5E6
:1028C800F7FFD5C5F8FF0900F5CF01F001502D0A33
:1028D800D1E0D3C5F6FFD4C5F7FFD5C5F8FF090089
:1028E800F5CF01F00150200ACCE0D3C5F6FFD4C5DE
:1028F800F7FFD5C5F8FF0900F5CF01F001502B0A05
:10290800C7E0D3C5F6FFD4C5F7FFD5C5F8FF090062
:10291800F5CF01F00150230AC2E0D3C5F6FFD4C5B4
:10292800F7FFD5C5F8FF0900F5CF01F00150300ACF
:10293800BDE001D09ED7E5A301D0E591E5A701D080
:10294800E595D3C5F6FFD4C5F7FFD5C5F8FF09004F
:10295800F5CF00F0000E016E00C00BF6D6EC0AF0C1
:10296800005238E00501E36BE46B0501E3C500F0B4
:10297800E4C501F00A0E046E000E056E25EC03F0A6
:10298800D3C5F6FFD4C5F7FFD5C5F8FF0900F5CFC5
:1029980002F002500024E36F000E0120E46F300EB5
:1029A800E35F000EE45B010ED327000ED423D5238A
:1029B800D3C5F6FFD4C5F7FFD5C5F8FF0900F5CF95
:1029C80000F0000E016E00C00BF6D6EC0AF00052C3
:1029D800CCE134D0D3C5F6FFD4C5F7FFD5C5F8FF91
:1029E8000900F5CF01F001502A0A28E1D6C5E9FF10
:1029F800D7C5EAFFEECF00F0EECF01F000C0E9FF47
:102A080001C0EAFFEECFE3F5EECFE4F5D6C5E9FF66
:102A1800D7C5EAFF020EEE24006E000EEE20016E0E
:102A2800D6C5E1FFD7C5E2FF00C0E6FF01C0E6FF5B
:102A3800010E0501D327000ED423D523D3C5F6FFF5
:102A4800D4C5F7FFD5C5F8FF0900F5CF01F001504F
:102A58002E0A72E10501010ED327000ED423D523D7
:102A6800D3C5F6FFD4C5F7FFD5C5F8FF0900F5CFE4
:102A780001F001502A0A28E1D6C5E9FFD7C5EAFFC7
:102A8800EECF00F0EECF01F000C0E9FF01C0EAFF91
:102A9800EECFE0F5EECFE1F5D6C5E9FFD7C5EAFF01
:102AA800020EEE24006E000EEE20016ED6C5E1FF88
:102AB800D7C5E2FF00C0E6FF01C0E6FF010ED3273D
:102AC800000ED423D52337D0E06BE16BD3C5F6FFD6
:102AD800D4C5F7FFD5C5F8FF0900F5CF00F0000E03
:102AE800016E00C00BF6D6EC0AF0005224E0E0C5F7
:102AF80000F0E1C501F00A0E046E000E056E25EC2B
:102B080003F0D3C5F6FFD4C5F7FFD5C5F8FF090014
:102B1800F5CF02F0025000240501E06F000E0120FD
:102B2800E16F300EE05F000EE15B010ED327000E6F
:102B3800D423D523CBD704D00501E06BE16BE6891C
:102B48000501D3C500F0D4C501F0D5C502F0010ECA
:102B5800D327000ED423D52300C0F6FF01C0F7FF0A
:102B680002C0F8FF0900F5CFE2F5F9D0F1C500F091
:102B7800F2C501F031EF24F0E589E2D7E6852ED1E0
:102B8800E58BE6812BD1E68329D1E58D27D126D1A6
:102B9800E58BE58F23D1D6C5E9FFD7C5EAFFEECF90
:102BA80000F0EECF01F000C0E9FF01C0EAFFEECF70
:102BB800EDF5EECFEEF5D6C5E9FFD7C5EAFF020E73
:102BC800EE24006E000EEE20016ED6C5E1FFD7C5DB
:102BD800E2FF00C0E6FF01C0E6FF000EEE1902E1C9
:102BE800000EED1904E1A00EED6F000EEE6FEF6B15
:102BF800F06BEF51ED25E96EF051EE21EA6EEE52E1
:102C08000BE0010EEF25006E000EF021016E00C0F2
:102C1800EFF501C0F0F5EDD7E051E1110AE0F05110
:102C2800E15D02E1EF51E05D04E2E0C5EFF5E1C5E9
:102C3800F0F5E451F05D02E1E351EF5D05E2EF519B
:102C4800E35FF051E45B02D0E36BE46BE5B716D0C9
:102C5800E3C500F0E4C501F0010EE35F000EE45B9C
:102C6800005001100BE0D1C5E1FFD2C5E2FF200EF4
:102C7800E66ED14BD22BF14BF22BEAD7EFC502F01F
:102C8800F0C503F0010EEF5D006E000EF059016E05
:102C980000C0EFF501C0F0F50250031019E0EDC5D2
:102CA800E9FFEEC5EAFFD1C5E1FFD2C5E2FFEECFED
:102CB800E6FFD14BD22B010EED25006E000EEE2162
:102CC800016E00C0EDF501C0EEF5F14BF22BD6D741
:102CD800E5A716D0E3C500F0E4C501F0010EE35FF7
:102CE800000EE45B005001100BE0D1C5E1FFD2C536
:102CF800E2FF200EE66ED14BD22BF14BF22BEAD736
:102D08008CD5D6C5E9FFD7C5EAFFEECF00F0EECFE8
:102D180001F000C0E9FF01C0EAFFEECFE2F5D6C539
:102D2800E9FFD7C5EAFF020EEE24006E000EEE2082
:102D3800016ED6C5E1FFD7C5E2FF00C0E6FF01C0BE
:102D4800E6FFE20EED6F050EEE6F010EEF6F000E5F
:102D5800F06F62D7C00EE513000EE6133FD0E251C4
:102D6800000AD8B403D7E2516C0AD8B405D7E251A7
:102D78004C0AD8B401D7E251660AD8B4FFD6E2515A
:102D8800450AD8B4FDD6E251650AD8B4FAD6E2515C
:102D9800670AD8B4F8D6E2516F0AD8B4F6D6E25129
:102DA800640AD8B4F4D6E251690AD8B4F0D6E2512C
:102DB800700AD8B4EDD6E251580AD8B4E9D6E2512F
:102DC800780AD8B4E6D6E251730AD8B4E4D6E25108
:102DD800630A97E0E251750ABDE0B3D7000EE51526
:102DE800006EE651070B016E00500110D8B4D4EF05
:102DF8001FF0E6A904D0060EE06F000EE16FD6C5FD
:102E0800E9FFD7C5EAFFEECF00F0EECF01F000C032
:102E1800E9FF01C0EAFFEECFE7F5EECFE8F5EECF28
:102E2800E9F5EECFEAF5D6C5E9FFD7C5EAFF040E06
:102E3800EE24006E000EEE20016ED6C5E1FFD7C568
:102E4800E2FF00C0E6FF01C0E6FF046A056A066A01
:102E5800076AE7C500F0E8C501F0E9C502F0EAC570
:102E680003F00BEC0BF0010ED8B0000E006E005210
:102E780005E0E97F030EE513000EE613EB6BEC6B40
:102E8800E7C500F0E8C501F0E9C502F0EAC503F0BE
:102E9800046A056A066A076A0FEC0EF0000ED8A4E9
:102EA800010E006E0052D8B48DD0EAC500F0016A58
:102EB800026A036AFF0E0016000E01167E0E005EFF
:102EC800000E015A00C0EBF501C0ECF5010E005EE2
:102ED800000E015A00C0EBF501C0ECF5030E046EBC
:102EE800000E056E25EC03F000C0EBF501C0ECF513
:102EF8000A0E046E000E056EABEC0DF000C0EBF58B
:102F080001C0ECF5800E0118026E800E025C02E131
:102F1800000E005C05E2010E0501EB5F000EEC5BA4
:102F28000501EB51000806010B6F26EC0EF0E7C512
:102F380004F0E8C505F0E9C506F0EAC507F020EC9D
:102F480007F000C0EDF501C0EEF502C0EFF503C0D3
:102F5800F0F5000E046E000E056E000E066E7F0E74
:102F6800076EEDC500F0EEC501F0EFC502F0F0C543
:102F780003F00BEC0BF0010ED8B0000E006E0052FF
:102F880006E0010E0501EB5F000EEC5B1BD0000EA6
:102F9800046E000E056E200E066E820E076EEDC5DD
:102FA80000F0EEC501F0EFC502F0F0C503F00BEC40
:102FB8000BF0000ED8B0010E006E005203E00501C0
:102FC800EB4BEC2B0501800E006E800EEC19005CBB
:102FD80002E1EB51000803E3010EE26F02D0EBC5FA
:102FE800E2F5E6B118D0E6A315D0800EEC19006E14
:102FF8007F0E005C02E1FC0EEB5D0BE3800EEC192A
:10300800006E800EE119005C02E1E051EB5D01E227
:1030180001D001D0F1D3E051E11106E0E6A304D0DC
:10302800010EE05F000EE15BE151000802E1E051B2
:10303800080803E2080EE26F02D0E0C5E2F5E7C532
:1030480000F0E8C501F0E9C502F0EAC503F0046A3A
:10305800056A066A076A0FEC0EF0000ED8A4010E86
:10306800006E0052D8B44CD1EBC50BF626EC0EF02E
:1030780000C004F001C005F002C006F003C007F06C
:10308800E7C500F0E8C501F0E9C502F0EAC503F0BC
:1030980018EC0AF000C0E7F501C0E8F502C0E9F550
:1030A80003C0EAF50501E251000806010B6F26ECA2
:1030B8000EF000C004F001C005F002C006F003C025
:1030C80007F0E7C500F0E8C501F0E9C502F0EAC578
:1030D80003F018EC0AF000C0F3F501C0F4F502C0E3
:1030E800F5F503C0F6F5F3C5E7F5F4C5E8F5F5C55C
:1030F800E9F5F6C5EAF5F3C500F0F4C501F0F5C544
:1031080002F0F6C503F072EC12F008EC11F000C002
:1031180004F001C005F002C006F003C007F0F3C5D3
:1031280000F0F4C501F0F5C502F0F6C503F004ECB3
:1031380011F0000E046E000E056E000E066E7E0E77
:10314800076E0BEC0BF0000ED8B0010E006E0052AB
:103158001AE0E7C500F0E8C501F0E9C502F0EAC5E4
:1031680003F0000E046E000E056E000E066E7E0E55
:10317800076E79EC04F000C0E7F501C0E8F502C07D
:10318800E9F503C0EAF5E7C500F0E8C501F0E9C5CF
:1031980002F0EAC503F072EC12F00501E251010FEA
:1031A800096E0A6A000E0A2209C004F00AC005F076
:1031B800000E0ABEFF0E066E076E04360490053632
:1031C8000636073604360490053606360736300EBE
:1031D8000424F66E890E0520F76E000E0620F86EA0
:1031E8000900F5CF05F00900F5CF06F00900F5CF85
:1031F80007F00900F5CF08F00850035C08E1075014
:10320800025C05E10650015C02E10550005C1EE32A
:103218000501E7C500F0E8C501F0E9C502F0EAC517
:1032280003F0CD0E046ECC0E056E4C0E066E7B0EB2
:10323800076E20EC07F000C0E7F501C0E8F502C012
:10324800E9F503C0EAF5EB4BEC2B5AD0E7C500F0E3
:10325800E8C501F0E9C502F0EAC503F072EC12F026
:10326800E2C504F0000E056E066E076E0436049083
:103278000536063607360436049005360636073610
:10328800300E0424F66E890E0520F76E000E062017
:10329800F86E0900F5CF05F00900F5CF06F0090032
:1032A800F5CF07F00900F5CF08F00850035C08E1F6
:1032B8000750025C05E10650015C02E10550005C24
:1032C8001FE20501E7C500F0E8C501F0E9C502F015
:1032D800EAC503F0000E046E000E056E200E066EA1
:1032E800820E076E20EC07F000C0E7F501C0E8F594
:1032F80002C0E9F503C0EAF5010EEB5F000EEC5BD6
:103308000501E6A394D0E6B792D0800E000A006EBD
:10331800800EE119005C02E1E0510A0804E20A0E9D
:10332800E06F000EE16FE7C500F0E8C501F0E9C500
:1033380002F0EAC503F072EC12F000C0EDF501C02E
:10334800EEF502C0EFF503C0F0F5ED51EE11EF1107
:10335800F01142E00A0E046E000E056E066E076E4E
:10336800EDC500F0EEC501F0EFC502F0F0C503F0C1
:1033780035EC0CF008C000F009C001F00AC002F0FA
:103388000BC003F0000E046E031808E10450021885
:1033980005E10450011802E10050000A1DE1010E88
:1033A800E05F000EE15B0A0E046E000E056E066E0D
:1033B800076EEDC500F0EEC501F0EFC502F0F0C5EF
:1033C80003F035EC0CF000C0EDF501C0EEF502C0DD
:1033D800EFF503C0F0F5B9D7800EE119006E800E45
:1033E800005C02E1E251E05D22E2E051E25D0601AB
:1033F8000B6F26EC0EF000C004F001C005F002C00F
:1034080006F003C007F0E7C500F0E8C501F0E9C51C
:1034180002F0EAC503F018EC0AF000C0E7F501C0B5
:10342800E8F502C0E9F503C0EAF5E0C5E2F5050EE6
:103438000501E025006E000EE121016E0050E35FFA
:103448000150E45BE051E11103E1E6B701D004D09B
:10345800010EE35F000EE45B030EE515006EE6C5A2
:1034680001F0000E01160050011004E0010EE35FA8
:10347800000EE45BE5A539D0E5A312D0E5A103D0A1
:103488002D0ED86F02D02B0ED86FD1C5E1FFD2C553
:10349800E2FFD8C5E6FFD14BD22BF14BF22B0CD073
:1034A800E5A10AD0D1C5E1FFD2C5E2FF200EE66E44
:1034B800D14BD22BF14BF22B800E006E800EE4190B
:1034C800005C02E1E35100080FE2D1C5E1FFD2C57B
:1034D800E2FF300EE66ED14BD22BF14BF22B010EF0
:1034E800E35F000EE45BE8D73AD0E5B718D0800E6A
:1034F800006E800EE419005C02E1E35100080FE25F
:10350800D1C5E1FFD2C5E2FF200EE66ED14BD22B2A
:10351800F14BF22B010EE35F000EE45BE8D7E5A365
:1035280012D0E5A103D02D0ED96F02D02B0ED96F82
:10353800D1C5E1FFD2C5E2FFD9C5E6FFD14BD22BF9
:10354800F14BF22B0CD0E5A10AD0D1C5E1FFD2C5D1
:10355800E2FF200EE66ED14BD22BF14BF22BE7C5E2
:1035680000F0E8C501F0E9C502F0EAC503F072EC25
:1035780012F000C0EDF501C0EEF502C0EFF503C092
:10358800F0F5E2C500F0000E016E026E036E003623
:1035980000900136023603360036009001360236B6
:1035A8000336300E0024F66E890E0120F76E000EE9
:1035B8000220F86E0900F5CF04F00900F5CF05F0F8
:1035C8000900F5CF06F00900F5CF07F0EDC500F0CA
:1035D800EEC501F0EFC502F0F0C503F035EC0CF0D4
:1035E800300E0026D1C5E1FFD2C5E2FF00C0E6FFDC
:1035F800D14BD22BF14BF22BE051E11103E1E6B7AD
:1036080001D06FD0D1C5E1FFD2C5E2FF2E0EE66E24
:10361800D14BD22BF14BF22BE251E05F000EE15B74
:10362800E2534DE0E207E2C500F0000E016E026EC3
:10363800036E0036009001360236033600360090DD
:10364800013602360336300E0024F66E890E01204C
:10365800F76E000E0220F86E0900F5CF04F009009D
:10366800F5CF05F00900F5CF06F00900F5CF07F012
:10367800EDC500F0EEC501F0EFC502F0F0C503F0AE
:1036880035EC0CF00A0E046E000E056E066E076E21
:1036980035EC0CF008C000F009C001F00AC002F0D7
:1036A8000BC003F0300E0026D1C5E1FFD2C5E2FF02
:1036B80000C0E6FFD14BD22BF14BF22BB1D7E05132
:1036C800E1110FE0D1C5E1FFD2C5E2FF300EE66E91
:1036D800D14BD22BF14BF22B010EE05F000EE15BD8
:1036E800EED7E5AB0BD0D1C5E1FFD2C5E2FF450E61
:1036F800E66ED14BD22BF14BF22B0AD0D1C5E1FFAC
:10370800D2C5E2FF650EE66ED14BD22BF14BF22B00
:10371800800EEC19006E800E005C02E1000EEB5D7D
:1037280011E2EB510008EB6FEC51000EEC57D1C5DC
:10373800E1FFD2C5E2FF2D0EE66ED14BD22BF14B45
:10374800F22B0AD0D1C5E1FFD2C5E2FF2B0EE66EFF
:10375800D14BD22BF14BF22B0A0E046E000E056EE4
:10376800EBC500F0ECC501F0ABEC0DF0300E002617
:10377800D1C5E1FFD2C5E2FF00C0E6FF0501D14B8C
:10378800D22BF14BF22B0A0E046E000E056EEBC520
:1037980000F0ECC501F0ABEC0DF008C000F009C07A
:1037A80001F0300E0026D1C5E1FFD2C5E2FF00C00E
:1037B800E6FF0501D14BD22BF14BF22BE5A71AD02E
:1037C800800E006E800EE419005C02E1E3510008EF
:1037D80011E2D1C5E1FFD2C5E2FF200EE66ED14B62
:1037E800D22BF14BF22B010EE35F000EE45BE351A9
:1037F800E411EFE111EF14F0E6A3F5D0800EEC1917
:10380800006E800E005C02E1000EEB5D0AE2010E24
:10381800EB5D006E000EEC59016E0050E05F015048
:10382800E15BE7C500F0E8C501F0E9C502F0EAC5CB
:1038380003F072EC12F000C0EDF501C0EEF502C025
:10384800EFF503C0F0F5010EE26FE2510A0A34E029
:10385800E2C500F0000E016E026E036E00360090A5
:10386800013602360336003600900136023603363A
:10387800300E0024F66E890E0120F76E000E02202D
:10388800F86E0900F5CF01F00900F5CF02F0090044
:10389800F5CF03F00900F5CF04F00450F05D08E11E
:1038A8000350EF5D05E10250EE5D02E10150ED5D70
:1038B80001E202D0E22BC9D7E251E05DF76F000EBA
:1038C800E159F86FF7C5E0F5F8C5E1F5EDC500F089
:1038D800EEC501F0EFC502F0F0C503F008EC11F0F9
:1038E80000C004F001C005F002C006F003C007F0F4
:1038F800E7C500F0E8C501F0E9C502F0EAC503F044
:1039080004EC11F000C0F3F501C0F4F502C0F5F5C0
:1039180003C0F6F5F7C50BF626EC0EF0F3C504F078
:10392800F4C505F0F5C506F0F6C507F020EC07F07C
:10393800000E046E000E056E000E066E7E0E076EFB
:1039480079EC04F072EC12F000C0EDF501C0EEF570
:1039580002C0EFF503C0F0F50501E051E11143E0C5
:103968000A0E046E000E056E066E076EEDC500F0B9
:10397800EEC501F0EFC502F0F0C503F035EC0CF030
:1039880008C000F009C001F00AC002F00BC003F043
:10399800000E046E031808E10450021805E10450F3
:1039A800011802E10050000A1EE105010A0E046E2A
:1039B800000E056E066E076EEDC500F0EEC501F04F
:1039C800EFC502F0F0C503F035EC0CF000C0EDF5E2
:1039D80001C0EEF502C0EFF503C0F0F5010EE05F9F
:1039E800000EE15BB9D70501800E006E800EE1196B
:1039F800005C02E1E0510C0816E3E0C50BF695EC1B
:103A080008F0E7C504F0E8C505F0E9C506F0EAC521
:103A180007F079EC04F000C0E7F501C0E8F502C052
:103A2800E9F503C0EAF5E7C500F0E8C501F0E9C526
:103A380002F0EAC503F0046A056A066A076A0FEC31
:103A48000EF0000ED8A4010E006E0052D8B478D043
:103A5800E7C500F0E8C501F0E9C502F0EAC503F0E2
:103A680072EC12F0000E046E031808E104500218FC
:103A780005E10450011802E10050000A61E1800EDE
:103A8800006E800E0501EC19005C02E1EB510108A3
:103A980057E2EBC50BF626EC0EF000C004F001C0AF
:103AA80005F002C006F003C007F0E7C500F0E8C55E
:103AB80001F0E9C502F0EAC503F018EC0AF05F0E60
:103AC800046E700E056E090E066E810E076E0BEC05
:103AD8000BF0010ED8B0000E006E005206E0090E81
:103AE8000501EB5F000EEC5B05D00501080EEB5FEE
:103AF800000EEC5BEBC50BF626EC0EF000C004F0F4
:103B080001C005F002C006F003C007F0E7C500F0E9
:103B1800E8C501F0E9C502F0EAC503F018EC0AF0BF
:103B280072EC12F000C0EDF501C0EEF502C0EFF541
:103B380003C0F0F50501E76BE86BE96BEA6B39D078
:103B48000501E7C500F0E8C501F0E9C502F0EAC5DE
:103B580003F072EC12F000C0EDF501C0EEF502C002
:103B6800EFF503C0F0F5EDC500F0EEC501F0EFC5C7
:103B780002F0F0C503F008EC11F000C004F001C039
:103B880005F002C006F003C007F0E7C500F0E8C57D
:103B980001F0E9C502F0EAC503F004EC11F000C039
:103BA800E7F501C0E8F502C0E9F503C0EAF5EB6BFB
:103BB800EC6B010EE26FE2510A0A34E0E2C500F054
:103BC800000E016E026E036E00360090013602365A
:103BD800033600360090013602360336300E0024D4
:103BE800F66E890E0120F76E000E0220F86E0900AD
:103BF800F5CF01F00900F5CF02F00900F5CF03F089
:103C08000900F5CF04F00450F05D08E10350EF5DC2
:103C180005E10250EE5D02E10150ED5D01E202D0E6
:103C2800E22BC9D7E251E025006E000EE121016EBA
:103C3800EB510026EC5101220050E35F0150E45B98
:103C4800E6B704D0E051E11101E104D0010EE35FD1
:103C5800000EE45B030EE515006EE6C501F0000EEC
:103C680001160050011004E0010EE35F000EE45B52
:103C7800E5A539D0E5A312D0E5A103D02D0EDA6F62
:103C880002D02B0EDA6FD1C5E1FFD2C5E2FFDAC54B
:103C9800E6FFD14BD22BF14BF22B0CD0E5A10AD089
:103CA800D1C5E1FFD2C5E2FF200EE66ED14BD22B83
:103CB800F14BF22B800E006E800EE419005C02E1DD
:103CC800E35100080FE2D1C5E1FFD2C5E2FF300E93
:103CD800E66ED14BD22BF14BF22B010EE35F000EB7
:103CE800E45BE8D73AD0E5B718D0800E006E800EB6
:103CF800E419005C02E1E35100080FE2D1C5E1FFDD
:103D0800D2C5E2FF200EE66ED14BD22BF14BF22B3F
:103D1800010EE35F000EE45BE8D7E5A312D0E5A14E
:103D280003D02D0EDB6F02D02B0EDB6FD1C5E1FF68
:103D3800D2C5E2FFDBC5E6FFD14BD22BF14BF22B0C
:103D48000CD0E5A10AD0D1C5E1FFD2C5E2FF200E13
:103D5800E66ED14BD22BF14BF22BE2C500F0E20715
:103D680000524CE0E2C500F0000E016E026E036ED8
:103D780000360090013602360336003600900136D0
:103D880002360336300E0024F66E890E0120F76ED7
:103D9800000E0220F86E0900F5CF04F00900F5CFF7
:103DA80005F00900F5CF06F00900F5CF07F0EDC5DD
:103DB80000F0EEC501F0EFC502F0F0C503F035ECF8
:103DC8000CF00A0E046E000E056E066E076E35ECDA
:103DD8000CF008C000F009C001F00AC002F00BC0E6
:103DE80003F0300E0026D1C5E1FFD2C5E2FF00C0C6
:103DF800E6FFD14BD22BF14BF22BAFD7800E006EE2
:103E0800800EEC19005C02E1EB5100080FE2D1C50D
:103E1800E1FFD2C5E2FF300EE66ED14BD22BF14B5B
:103E2800F22B010EEB5F000EEC5BE8D7800E000A68
:103E3800006E800EE119005C02E1E051080803E21F
:103E4800080EE26F02D0E0C5E2F5E251E05F000E35
:103E5800E15BE25303E1E6B701D00AD0D1C5E1FF47
:103E6800D2C5E2FF2E0EE66ED14BD22BF14BF22BD0
:103E7800E2C50BF626EC0EF0E7C504F0E8C505F040
:103E8800E9C506F0EAC507F020EC07F072EC0BF084
:103E980000C0EDF501C0EEF502C0EFF503C0F0F586
:103EA8000501E2534DE0E207E2C500F0000E016EA5
:103EB800026E036E00360090013602360336003675
:103EC8000090013602360336300E0024F66E890E55
:103ED8000120F76E000E0220F86E0900F5CF04F0FD
:103EE8000900F5CF05F00900F5CF06F00900F5CF78
:103EF80007F0EDC500F0EEC501F0EFC502F0F0C522
:103F080003F035EC0CF00A0E046E000E056E066E1A
:103F1800076E35EC0CF008C000F009C001F00AC0CB
:103F280002F00BC003F0300E0026D1C5E1FFD2C568
:103F3800E2FF00C0E6FFD14BD22BF14BF22BB0D7FA
:103F4800E051E1110FE0D1C5E1FFD2C5E2FF300E2B
:103F5800E66ED14BD22BF14BF22B010EE05F000E37
:103F6800E15BEED7E5A71AD0800E006E800EE4194B
:103F7800005C02E1E351000811E2D1C5E1FFD2C5BE
:103F8800E2FF200EE66ED14BD22BF14BF22B010E45
:103F9800E35F000EE45BE351E411EFE111EF14F08D
:103FA800C00EE515016EE6C502F0000E0216000E01
:103FB800021802E1000E0118D8A480D0E5A927D084
:103FC800D6C5E9FFD7C5EAFFEECF00F0EECF01F086
:103FD80000C0E9FF01C0EAFFEECFEDF5EECFEEF548
:103FE800EECFEFF5EECFF0F5D6C5E9FFD7C5EAFF7E
:103FF800040EEE24006E000EEE20016ED6C5E1FF21
:10400800D7C5E2FF00C0E6FF01C0E6FF2FD0D6C546
:10401800E9FFD7C5EAFFEECF00F0EECF01F000C010
:10402800E9FF01C0EAFFEECF00F0EECF01F0000E8D
:1040380001BEFF0E026E036E00C0EDF501C0EEF585
:1040480002C0EFF503C0F0F5D6C5E9FFD7C5EAFF12
:10405800020EEE24006E000EEE20016ED6C5E1FFC2
:10406800D7C5E2FF00C0E6FF01C0E6FF800EF019E9
:10407800006E800E005C08E1000EEF5D05E1000EA9
:10408800EE5D02E1000EED5D18E2030EE513000E91
:10409800E613006A016A026A036AED51005EEE5196
:1040A800015AEF51025AF051035A00C0EDF501C010
:1040B800EEF502C0EFF503C0F0F54ED0E5A927D024
:1040C800D6C5E9FFD7C5EAFFEECF00F0EECF01F085
:1040D80000C0E9FF01C0EAFFEECFEDF5EECFEEF547
:1040E800EECFEFF5EECFF0F5D6C5E9FFD7C5EAFF7D
:1040F800040EEE24006E000EEE20016ED6C5E1FF20
:10410800D7C5E2FF00C0E6FF01C0E6FF25D0D6C54F
:10411800E9FFD7C5EAFFEECF00F0EECF01F000C00F
:10412800E9FF01C0EAFFEECFEDF5EECFEEF5000EA8
:10413800EF6FF06FD6C5E9FFD7C5EAFF020EEE2490
:10414800006E000EEE20016ED6C5E1FFD7C5E2FF76
:1041580000C0E6FF01C0E6FF000EE11902E1000E13
:10416800E0190FE1000E006EF01908E10050EF1998
:1041780005E10050EE1902E1ED51000A02E1E04BC1
:10418800E12BC00EE515006E00C005F0AED0010EA3
:10419800E26FE2510A0A34E0E2C500F0000E016E57
:1041A800026E036E00360090013602360336003682
:1041B8000090013602360336300E0024F66E890E62
:1041C8000120F76E000E0220F86E0900F5CF01F00D
:1041D8000900F5CF02F00900F5CF03F00900F5CF8B
:1041E80004F00450F05D08E10350EF5D05E1025072
:1041F800EE5D02E10150ED5D01E202D0E22BC9D78C
:1042080082D0010EE26FE251080A34E0E2C500F004
:10421800000E016E026E036E003600900136023603
:10422800033600360090013602360336350E002478
:10423800F66E8A0E0120F76E000E0220F86E090055
:10424800F5CF01F00900F5CF02F00900F5CF03F032
:104258000900F5CF04F00450F05D08E10350EF5D6C
:1042680005E10250EE5D02E10150ED5D01E202D090
:10427800E22BC9D748D0010EE26FE2510C0A34E0B4
:10428800E2C500F0000E016E026E036E003600906B
:104298000136023603360036009001360236033600
:1042A800030E0024F66E880E0120F76E000E022021
:1042B800F86E0900F5CF01F00900F5CF02F009000A
:1042C800F5CF03F00900F5CF04F00450F05D08E1E4
:1042D8000350EF5D05E10250EE5D02E10150ED5D36
:1042E80001E202D0E22BC9D70ED00550000AD8B49B
:1042F8004ED70550C00AD8B44AD70550800A81E085
:104308000550400AB8E0800E006E800EE119005C8E
:1043180002E1E051E25D03E2E0C5E2F50DD0800E76
:10432800E119006E800E005C02E1E251E05D04E2FA
:10433800E2C5E0F5000EE16FE351E4110EE0030E73
:10434800E515006EE6C501F0000E011600500110DB
:1043580004E0010EE35F000EE45B800EE119006EDD
:10436800800EE419005C02E1E351E05D05E2E051F2
:10437800E35FE151E45B02D0E36BE46BC40EE51547
:10438800016EE651080B026E0250080A02E1400E67
:10439800011808E1E351E41104E0010EE35F000EA7
:1043A800E45B1CD0C00EE515016EE651080B026EE9
:1043B8000250080A02E1800E011810E1800E006E1A
:1043C800800EE419005C02E1E351020805E2020EE6
:1043D800E35F000EE45B02D0E36BE46BE5A55DD020
:1043E800E5A312D0E5A103D02D0EDC6F02D02B0E71
:1043F800DC6FD1C5E1FFD2C5E2FFDCC5E6FFD14BDA
:10440800D22BF14BF22B34D0E5A10BD0D1C5E1FF73
:10441800D2C5E2FF200EE66ED14BD22BF14BF22B28
:1044280027D0C00EE515016EE651080B026E02504A
:10443800080A02E1800E01181BE1D1C5E1FFD2C5CF
:10444800E2FF300EE66ED14BD22BF14BF22BE5ABEF
:1044580003D0580EDD6F02D0780EDD6FD1C5E1FFB5
:10446800D2C5E2FFDDC5E6FFD14BD22BF14BF22BD3
:10447800E351E41111E0D1C5E1FFD2C5E2FF300EEE
:10448800E66ED14BD22BF14BF22B010EE35F000EFF
:10449800E45BE351E411EFE174D0E351E41113E07C
:1044A800E5B711D0D1C5E1FFD2C5E2FF200EE66E17
:1044B800D14BD22BF14BF22B010EE35F000EE45BE4
:1044C800E351E411EFE1E5A312D0E5A103D02D0EED
:1044D800DE6F02D02B0EDE6FD1C5E1FFD2C5E2FF41
:1044E800DEC5E6FFD14BD22BF14BF22B0CD0E5A168
:1044F8000AD0D1C5E1FFD2C5E2FF200EE66ED14B4E
:10450800D22BF14BF22BC00EE515016EE651080BCC
:10451800026E0250080A02E1400E01180BE1D1C5F3
:10452800E1FFD2C5E2FF300EE66ED14BD22BF14B44
:10453800F22B27D0C00EE515016EE651080B026E6E
:104548000250080A02E1800E01181BE1D1C5E1FF03
:10455800D2C5E2FF300EE66ED14BD22BF14BF22BD7
:10456800E5AB03D0580EDF6F02D0780EDF6FD1C5F0
:10457800E1FFD2C5E2FFDFC5E6FFD14BD22BF14BFD
:10458800F22B800E006E800EE119005C02E1E05112
:10459800E25D0BE2D1C5E1FFD2C5E2FF300EE66E67
:1045A800D14BD22BF14BF22BECD7E0C500F0E1C593
:1045B80001F0010EE05F000EE15B00500110D8B47D
:1045C8002AD1C00EE515006E00C0F3F50AD1E0C58A
:1045D80000F0E1C501F0000EE1BFFF0E026E036EB0
:1045E8000036009001360236033600360090013658
:1045F80002360336300E0024F66E890E0120F76E5F
:10460800000E0220F86E0900F5CF04F00900F5CF7E
:1046180005F00900F5CF06F00900F5CF07F0EDC564
:1046280000F0EEC501F0EFC502F0F0C503F035EC7F
:104638000CF00A0E046E000E056E066E076E35EC61
:104648000CF008C000F009C001F00AC002F00BC06D
:1046580003F0300E0024E26FD3D0E5AB45D0E0C5BF
:1046680000F0E1C501F0000EE1BFFF0E026E036E1F
:1046780000360090013602360336003600900136C7
:1046880002360336350E0024F66E8A0E0120F76EC8
:10469800000E0220F86E0900F5CF04F00900F5CFEE
:1046A80005F00900F5CF06F00900F5CF07F0EDC5D4
:1046B80000F0EEC501F0EFC502F0F0C503F035ECEF
:1046C8000CF00F0E0016000E011602160316560EF9
:1046D8000024F66E8C0E0120F76E000E0220F86E94
:1046E8000900F5CFE2F544D0E0C500F0E1C501F0DE
:1046F800000EE1BFFF0E026E036E00360090013619
:104708000236033600360090013602360336350E7F
:104718000024F66E8A0E0120F76E000E0220F86E55
:104728000900F5CF04F00900F5CF05F00900F5CF31
:1047380006F00900F5CF07F0EDC500F0EEC501F071
:10474800EFC502F0F0C503F035EC0CF00F0E0016C3
:10475800000E011602160316670E0024F66E8C0E64
:104768000120F76E000E0220F86E0900F5CFE2F581
:1047780047D0E0C500F0E1C501F0000EE1BFFF0E33
:10478800026E036E0036009001360236033600369C
:104798000090013602360336030E0024F66E880EAA
:1047A8000120F76E000E0220F86E0900F5CF04F024
:1047B8000900F5CF05F00900F5CF06F00900F5CF9F
:1047C80007F0EDC500F0EEC501F0EFC502F0F0C549
:1047D80003F035EC0CF0070E0014E26F300EE22700
:1047E8000FD0F351000AD8B4F2D6F351C00AD8B4A6
:1047F800EED6F351800AD8B430D7F351400AB9E065
:10480800D1C5E1FFD2C5E2FFE2C5E6FFD14BD22B0D
:10481800F14BF22BCAD6E5A71AD0800E006E800E97
:10482800E419005C02E1E351000811E2D1C5E1FF9F
:10483800D2C5E2FF200EE66ED14BD22BF14BF22B04
:10484800010EE35F000EE45BE351E411EFE111EFC9
:0C48580014F0F1C500F0F2C501F01200F0
:10486400D3C5F6FFD4C5F7FFD5C5F8FF0900F5CFCA
:1048740000F0005218E0D3C5F6FFD4C5F7FFD5C544
:10488400F8FF0900F5CF00F0D1C5E1FFD2C5E2FF82
:1048940000C0E6FF0501D14BD22B010ED327000E39
:1048A400D423D523DDD7D1C5E1FFD2C5E2FFE66A23
:0248B4001200F0
:1048B6000501D46B030ED45D0AE2D451D225E16E14
:1048C600000ED321E26E200EE66ED42BF3D7D45120
:1048D600D225E16E000ED321E26EE66AD407D451EA
:1048E600D225D56F000ED321D66F0A0E046ED1C520
:1048F60000F0ECEC06F008C000F0300E0026D5C53E
:10490600E1FFD6C5E2FF00C0E6FF0A0E046ED1C580
:1049160000F0ECEC06F000C0D1F50050000A01E111
:0849260002D0D407DCD7120017
:10492E000501D551D12506010B6FD2C50CF6D5C5A3
:10493E0000F00036009000500501D35D06010D6FAA
:10494E00D4C50EF628EC13F00501D351D12506017E
:10495E000B6F0C6B000E0C230501D55106010B5F7E
:10496E00000E0C5B010E0B5F000E0C5B0501D551AA
:10497E00D22506010D6F0E6B000E0E23D5C50FF658
:10498E00000E106F010E116FD5C500F0000E016EF6
:10499E0000360136009000500501D45D0601126FFD
:1049AE0001C013F6000E1357010E125F000E135BBB
:1049BE0002EC08F00501D551D12506010B6F0C6BE9
:1049CE00000E0C230501D551D22506010D6F0E6B7D
:1049DE00000E0E23D5C50FF6000E106F020E116FCE
:1049EE00D5C500F0000E016E003601360090005065
:1049FE000501D45D0601126F01C013F6000E1357A8
:0E4A0E00010E125F000E135B02EC08F01200A6
:104A1C00D1C521F6000E0601226FD2C523F6000E79
:104A2C00246FD3C525F6000E266FD4C527F6000ECD
:104A3C00286FCAEC01F0D3C521F6000E226FD4C545
:104A4C0023F6000E246FD5C525F6000E266FD6C5AD
:104A5C0027F6000E286FCAEC01F0D5C521F6000E22
:104A6C00226FD6C523F6000E246FD1C525F6000E95
:104A7C00266FD2C527F6000E286FCAEC01F0120083
:104A8C000501D151D55DF56FD251D659F66FD35181
:104A9C00D75DF76FD451D859F86FD151D95DF96FF3
:104AAC00D251DA59FA6FD351DB5DFB6FD451DC591B
:104ABC00FC6FD551D95DFD6FD651DA59FE6FD751C8
:104ACC00DB5D0601016F0501D851DC590601026F4F
:104ADC00036B046B056B066B076B086B096B0A6B3E
:104AEC000501D451D85D02E1D351D75D18E2D3C58D
:104AFC00DDF5D4C5DEF5D7C5D3F5D8C5D4F5DDC500
:104B0C00D7F5DEC5D8F5D1C5DFF5D2C5E0F5D5C5ED
:104B1C00D1F5D6C5D2F5DFC5D5F5E0C5D6F5D8515A
:104B2C00DC5D02E1D751DB5D18E2DBC5E1F5DCC5EC
:104B3C00E2F5D7C5DBF5D8C5DCF5E1C5D7F5E2C59F
:104B4C00D8F5D9C5E3F5DAC5E4F5D5C5D9F5D6C59B
:104B5C00DAF5E3C5D5F5E4C5D6F5D451D85D02E157
:104B6C00D351D75D18E2D3C5E5F5D4C5E6F5D7C565
:104B7C00D3F5D8C5D4F5E5C5D7F5E6C5D8F5D1C577
:104B8C00E7F5D2C5E8F5D5C5D1F5D6C5D2F5E7C55B
:104B9C00D5F5E8C5D6F5D451DC1902E1DB51D319B2
:104BAC003EE1D1C5EFF5D2C5F0F5D1C5EDF5D2C5D5
:104BBC00EEF5D251D65D02E1D151D55D05E2D5C5F8
:104BCC00EDF5D6C5EEF50AD0D651F05D02E1D55122
:104BDC00EF5D04E2D5C5EFF5D6C5F0F5EE51DA5D23
:104BEC0002E1ED51D95D05E2D9C5EDF5DAC5EEF579
:104BFC000AD0DA51F05D02E1D951EF5D04E2D9C57A
:104C0C00EFF5DAC5F0F5EDC50BF6D3C50CF6ED51A5
:104C1C00EF5D06010D6F0D2B0EEC13F057D1050156
:104C2C00D851DC1902E1DB51D71905E1D7C5F3F5F1
:104C3C00D8C5F4F506D0010ED75DF36F000ED85928
:104C4C00F46FD3C5F1F5D4C5F2F5800EF419006EEE
:104C5C00800EF219005C02E1F151F35DD8A082D014
:104C6C00F7C504F0F8C505F0000EF8BFFF0E066E90
:104C7C00076E03C600F004C601F005C602F006C6B6
:104C8C0003F01BEC11F00501D1510024FF6FD25140
:104C9C0001200601006FFFC5EDF500C6EEF5FBC562
:104CAC0004F0FCC505F0000E0501FCBFFF0E066EFE
:104CBC00076E07C600F008C601F009C602F00AC666
:104CCC0003F01BEC11F00501D1510024046ED251FC
:104CDC000120056E04C0EFF505C0F0F5F551060195
:104CEC0003270501F65106010423000E0501F6BF4A
:104CFC00FF0E0601052306230501F95106010727BE
:104D0C000501FA5106010823000E0501FABFFF0E3A
:104D1C00060109230A23800E0518006E800E001967
:104D2C00005C03E10501FF51045C0CE2EDC5E9F503
:104D3C00EEC5EAF5EFC5EDF5F0C5EEF5E9C5EFF515
:104D4C00EAC5F0F50501EDC50BF6F1C50CF6ED5114
:104D5C00EF5D06010D6F0D2B0EEC13F00501F14B01
:104D6C00F22B73D7D751F15D006ED851F259016E09
:104D7C00FDC504F0FEC505F025EC03F000C003F6FC
:104D8C0001C004F6000E0601056F066F0501D35134
:104D9C00F15D006ED451F259016EF9C504F0FAC5FB
:104DAC0005F025EC03F000C007F601C008F6000E74
:104DBC000601096F0A6F0501F251DC5D02E1F15148
:104DCC00DB5DD8A083D001C604F002C605F0000E4E
:104DDC00060102BFFF0E066E076E03C600F004C686
:104DEC0001F005C602F006C603F01BEC11F005013C
:104DFC00D5510024FF6FD65101200601006FFFC56D
:104E0C00EDF500C6EEF5FBC504F0FCC505F0000E93
:104E1C000501FCBFFF0E066E076E07C600F008C644
:104E2C0001F009C602F00AC603F01BEC11F00501F3
:104E3C00D1510024046ED2510120056E04C0EFF54F
:104E4C0005C0F0F5FD51060103270501FE510601D1
:104E5C000423000E0501FEBFFF0E060105230623E9
:104E6C000501F951060107270501FA51060108232E
:104E7C00000E0501FABFFF0E060109230A23800E5E
:104E8C000518006E800E0019005C03E10501FF514E
:104E9C00045C0CE2EDC5EBF5EEC5ECF5EFC5EDF5FC
:104EAC00F0C5EEF5EBC5EFF5ECC5F0F50501EDC57C
:104EBC000BF6F1C50CF6ED51EF5D06010D6F0D2BE8
:0E4ECC000EEC13F00501F14BF22B75D712001E
:104EDA000501D5510108D76FD6C5D8F5000ED857A8
:104EEA00010EDD6F000EDE6FFE0E006EFF0E016E0C
:104EFA00D5C504F0D6C505F025EC03F000C0D9F5F8
:104F0A0001C0DAF5DF6BE06BD5C5DBF5D6C5DCF59C
:104F1A00D1C539F6D551D32506013A6F1BEC00F0FD
:104F2A00D1C539F60501D551D35D06013A6F1BEC9F
:104F3A0000F00501D551D1250601396FD3C53AF6DE
:104F4A001BEC00F00501D551D15D0601396FD3C5BF
:104F5A003AF61BEC00F0800E0501E019006E800E97
:104F6A00DC19005C02E1DB51DF5DD8B08BD0800E2A
:104F7A00D819006E800E005C02E1000ED75D12E3C4
:104F8A00010EDB5F000EDC5B020ED925006E000EFF
:104F9A00DA21016E00C0D9F501C0DAF50050D72731
:104FAA000150D823DF4BE02B020EDD25006E000EE8
:104FBA00DE21016E00C0DDF501C0DEF50050D72705
:104FCA000150D823DF51D1250601396F0501DB5184
:104FDA00D32506013A6F1BEC00F00501DF51D15DC4
:104FEA000601396F0501DB51D32506013A6F1BEC27
:104FFA0000F00501DF51D1250601396F0501DB51AA
:10500A00D35D06013A6F1BEC00F00501DF51D15D5B
:10501A000601396F0501DB51D35D06013A6F1BECBE
:10502A0000F00501DB51D1250601396F0501DF5179
:10503A00D32506013A6F1BEC00F00501DB51D15D67
:10504A000601396F0501DF51D32506013A6F1BECC2
:10505A0000F00501DB51D1250601396F0501DF5149
:10506A00D35D06013A6F1BEC00F00501DB51D15DFF
:10507A000601396F0501DF51D35D06013A6F1BEC5A
:06508A0000F069D71200DE
:10509000D1C51EF60501D551D35D06011F6FD5C5DB
:1050A00020F620372091202B9AEC06F0D1C50BF684
:1050B000D2C50CF6D3C50DF6D4C50EF6D5C50FF680
:1050C000D6C510F6030E116F126B136B02EC08F0CD
:0250D0001200CC
:1050D2000501D551D12506010B6FD2C50CF6D5C5F8
:1050E20000F00036009000500501D35D06010D6FFF
:1050F2000EEC13F00501D551D12506010B6F050108
:10510200D451D22506010C6F020E0C5FD5C500F0FA
:105112000036009000500501D35D06010D6F0EECC4
:1051220013F0D1C51EF60501D551D22506011F6F18
:10513200D5C500F00036009000500501D45D06018F
:10514200206F9AEC06F00501D351D12506011E6F9E
:105152001E070501D551D22506011F6FD5C500F0E6
:105162000036009000500501D45D0601206F9AECD4
:1051720006F00501D551D12506010B6F0C6B000E0F
:105182000C230501D551D22506010D6F0E6B000EC1
:105192000E23D5C50FF6000E106F010E116FCAEC6B
:1051A20011F00501D351D12506010B6F0C6B000ED6
:1051B2000C230501D55106010B5F000E0C5B010E9D
:1051C2000B5F000E0C5B0501D551D22506010D6F58
:1051D2000E6B000E0E23D5C50FF6000E106F020ED9
:1051E200116FCAEC11F00501D351D12506010B6FE5
:1051F2000C6B000E0C230501D55106010B5F000E4E
:105202000C5B010E0B5F000E0C5B0501D451D22525
:1052120006010D6F0E6B000E0E230501D55106011E
:105222000D5F000E0E5B010E0D5F000E0E5BD5C50D
:105232000FF6000E106F040E116FCAEC11F005018B
:10524200D551D12506010B6F0C6B000E0C23050105
:10525200D451D22506010D6F0E6B000E0E230501EF
:10526200D55106010D5F000E0E5B010E0D5F000EA3
:105272000E5BD5C50FF6000E106F080E116FCAEC4B
:0452820011F0120015
:10528600016A026A040E025C02E1000E015C0AE297
:10529600580E0124E16E010E0220E26EE66A014A12
:0652A600022AF0D71200FD
:1052AC00270E06010B6F0BEC0CF006010B6B0BECD5
:1052BC000CF0D1C50BF60BEC0CF006010B6B0BECE8
:1052CC000CF0D2C50BF60BEC0CF006010B6B0BECD7
:1052DC000CF0FF0E06010B6F0BEC0CF02F0E060101
:0852EC000B6F0BEC0CF012003B
:1052F400A30E06010B6F0BEC0CF006010B6B0BEC11
:105304000CF0400E06010B6F0BEC0CF0290E06019D
:105314000B6F0BEC0CF006010B6B0BEC0CF0D1C516
:105324000BF60BEC0CF006010B6B0BEC0CF0D2C57E
:105334000BF60BEC0CF0010E06010B6F0BEC0CF0F2
:0C5344002F0E06010B6F0BEC0CF012009A
:10535000A30E06010B6F0BEC0CF006010B6B0BECB4
:105360000CF0400E06010B6F0BEC0CF02A0E060140
:105370000B6F0BEC0CF006010B6B0BEC0CF0D1C5BA
:105380000BF60BEC0CF006010B6B0BEC0CF0D2C522
:105390000BF60BEC0CF0010E06010B6F0BEC0CF096
:0C53A0002F0E06010B6F0BEC0CF012003E
:1053AC00800E0501D15D04E2400ED25D01E201D018
:0C53BC0004D0D1C59AF0D2C519F012003F
:1053C8000501D66BD76BD86BD96BDA6BDB6BD1C5A4
:1053D800DAF5D2C5DBF5D1C50BF6D2C50CF645EC2E
:1053E80013F045D10501D851D325E96E000ED4211B
:1053F800EA6EEE50000A67E0080EDB5D64E2D85101
:10540800D325E96E000ED421EA6E200EEE5CD66F2D
:10541800DA51780809E2D1C5DAF5DB2BD1C50BF6EC
:10542800DBC50CF645EC13F00501D76B060ED75D0E
:1054380046E2060E006E000E016E026E036ED6C5C1
:1054480004F0000E056E066E076EE2EC0AF0BC0E64
:1054580000267A0E0122000E0222D7510024F66E91
:10546800000E0120F76E000E0220F86E0900F5CF3D
:1054780000F000C0D9F500C00BF67EEC13F0070E63
:10548800026EDBC500F0000E016E025005E000362A
:1054980000900136FF0FFAD70501DA510026000EF9
:1054A8000122D7510026000E0122580E0024E16E79
:1054B800010E0120E26ED9C5E6FFD72BB7D7060E3D
:1054C800DA27D82B8FD7DDD0D3C50BF6D4C50CF689
:1054D80061EC13F00501D86BD851D325E96E000EA5
:1054E800D421EA6EEE50000AD8B4BFD0100ED85DB1
:1054F800D8B0BBD0D851D325E96E000ED421EA6EBE
:10550800200EEE5CD66FDAC50BF6DBC50CF645EC63
:1055180013F00501D76B080ED75D46E2040E026E44
:10552800D6C500F0000E016E025005E0003600906E
:105538000136FF0FFAD7D7510026000E0122CC0EF4
:105548000024F66E6C0E0120F76E000EF86E000E49
:1055580001BEFF0EF8220900F5CF00F000C0D9F512
:1055680000C00BF67EEC13F0070E026EDBC500F0F0
:10557800000E016E025005E0003600900136FF0F64
:10558800FAD70501DA510026000E0122D75100266C
:10559800000E0122580E0024E16E010E0120E26E79
:1055A800D9C5E6FFD72BB7D7DAC50BF6DB51010F04
:1055B80006010C6F45EC13F00501D76B080ED75D9B
:1055C80050E2040E026ED6C500F0000E016E0250C5
:1055D80005E0003600900136FF0FFAD7D7510026B4
:1055E800000E0122080E0026000E0122CC0E002417
:1055F800F66E6C0E0120F76E000EF86E000E01BEFE
:10560800FF0EF8220900F5CF00F000C0D9F500C060
:105618000BF67EEC13F00501DB51010F036E046AF3
:10562800000E0422070E026E03C000F004C001F051
:10563800025005E0003600900136FF0FFAD7DA5124
:105648000026000E0122D7510026000E0122580E16
:105658000024E16E010E0120E26ED9C5E6FFD72BCA
:10566800ADD7080EDA27D82B37D70BD00AD00501CB
:10567800D551010AD8B4B6D6D551020AD8B424D720
:04568800F5D7120040
:10568C00260E06010B6F0BEC0CF006010B6B0BECF2
:10569C000CF0D1C50BF60BEC0CF006010B6B0BEC04
:1056AC000CF0D2C50BF60BEC0CF006010B6B0BECF3
:1056BC000CF0FF0E06010B6F0BEC0CF02F0E06011D
:0856CC000B6F0BEC0CF0120057
:0C56D4002E0E06010B6F0BEC0CF0120008
:0A56E0000AEC0AF00AEC0AF01200CE
:1056EA00210E06010B6F0BEC0CF006010B6B0BEC99
:1056FA000CF07F0E06010B6F0BEC0CF0220E06016C
:10570A000B6F0BEC0CF006010B6B0BEC0CF0070E9D
:10571A0006010B6F0BEC0CF00501D16BD26B800EFE
:10572A00D219006E800E040A005C02E1000ED15DFF
:10573A0028E276EC02F02DC121F6C0EC02F0400E10
:10574A000601216FC0EC02F00501D36B100ED35D88
:10575A000FE2580ED125E96E010ED221EA6EEECF84
:10576A0021F6C0EC02F00501D14BD22BD32BEED798
:10577A00010ED15F000ED25BBEEC02F0D14BD22BF0
:04578A00CED7120064
:10578E000A0E0101366F010E376F000E386F000ED4
:10579E00396FEC0E3A6F040E3B6F000E3C6F000E2D
:1057AE003D6FFF0E4A6FFF0E4B6F000E4C6F000EDB
:1057BE004D6FFF0E4E6FFF0E4F6FFF0E506FFF0EB1
:1057CE00516F800E426F050E436F210E446F060E11
:1057DE00456F7C0E466F050E476F000E486F000E2C
:1057EE00496F949894968B988B9694889486C79EBE
:0857FE00C79C380EC66E1200B4
:1058060071DF150E0C6EC60E0D6E0D2EFED70C2E0C
:10581600FCD70000A30E06010B6F0BEC0CF0060183
:105826000B6B0BEC0CF0400E06010B6F0BEC0CF047
:1058360006010B6B0BEC0CF0C1C50BF60BEC0CF078
:1058460006010B6B0BEC0CF0C2C50BF60BEC0CF067
:1058560006010B6B0BEC0CF0010E06010B6F0BEC4B
:105866000CF02F0E06010B6F0BEC0CF036DF2FDF62
:0258760012001E
:105878000501BC6B76EC02F0C1C521F6C0EC02F064
:105888000050000A06E02E0E06013B6F0EEC00F0F9
:105898003DD066C5D1F567C5D2F55C0E0501D36F5D
:1058A8008B0ED46F000ED56F32EC24F066C50BF664
:1058B80067C50CF661EC13F000C060F501C061F536
:1058C800C1C5D1F5680E0501D26F050ED36F5BEC2B
:1058D80024F060516625D16F61516721D26F680E3F
:1058E800D36F050ED46FA3EC13F066C5D1F567C569
:1058F800D2F5D3EC13F0780ED16F8C0ED26F000E68
:10590800D36FEEEC13F0010E0501BC6FBEEC02F094
:06591800BCC500F0120006
:10591E00B3DC320E0501D16F080ED26F40DD680E7A
:10592E00D16F050ED26FA10ED36F8C0ED46F000EF9
:10593E00D56F32EC24F0320E0501D16F020ED26F0C
:10594E00680ED36F050ED46F010ED56F36DDC6DE31
:10595E00150E0C6EC60E0D6E0D2EFED70C2EFCD730
:10596E000000D16B0F0ED26F8ADE0AEC0AF0ABDEAE
:10597E000AEC0AF00501D16B0F0ED26F90DC0AEC27
:10598E000AF0A1DE0AEC0AF00501D16B070ED26F08
:10599E00AADC0AEC0AF00501D16B070ED26FD1DC3E
:0859AE000AEC0AF090DE120081
:1059B6000501C15306E0A70E06010B6F0BEC0CF0B8
:0E59C60005D0A60E06010B6F0BEC0CF01200C4
:1059D4000501C76BC86B000EC85D02E10A0EC75D06
:1059E4000BE2C751C525E16EC851C621E26E200EF7
:1059F400E66EC74BC82BEFD7C751C525E16EC8511A
:105A0400C621E26EE66A010EC75F000EC85BC7518D
:105A1400C525C96FC851C621CA6F0A0E046E000E8F
:105A2400056E066E076EC1C500F0C2C501F0C3C5A0
:105A340002F0C4C503F035EC0CF008C000F009C056
:105A440001F00AC002F00BC003F0300E0026C9C5F5
:105A5400E1FFCAC5E2FF00C0E6FF0A0E046E000EB5
:105A6400056E066E076EC1C500F0C2C501F0C3C560
:105A740002F0C4C503F035EC0CF000C0C1F501C060
:105A8400C2F502C0C3F503C0C4F5000E046E0318CA
:105A940008E10450021805E10450011802E1005025
:105AA400000A01E105D0010EC75F000EC85BAFD745
:025AB4001200DE
:105AB600C60E0501CC6F050ECD6FC1C5D1F5C2C5A9
:105AC600D2F5C3C5D3F5C4C5D4F5C5C5D5F5CC0E39
:105AD600D66F050ED76F0CEC14F000C0CAF501C0E6
:105AE600CBF50050C125E16E0150C221E26EE66A97
:0A5AF600CAC500F0CBC501F0120094
:105B0000AE0E06010B6F0BEC0CF0110E0B6E3C0E83
:105B10000C6ECB0E0D6E0D2EFED70C2EFCD70B2E61
:105B2000FAD7AF0E06010B6F0BEC0CF0090E0B6EE3
:105B30001E0E0C6EE40E0D6E0D2EFED70C2EFCD735
:105B40000B2EFAD70000B00E06010B6F0BEC0CF019
:105B500006010B6B0BEC0CF0100E06010B6F0BEC3F
:105B60000CF0200E06010B6F0BEC0CF006010B6B1A
:105B70000BEC0CF0210E06010B6F0BEC0CF0060188
:105B80000B6B0BEC0CF07F0E06010B6F0BEC0CF0AB
:105B9000220E06010B6F0BEC0CF006010B6B0BECED
:105BA0000CF0070E06010B6F0BEC0CF0A10E0601BA
:105BB0000B6F0BEC0CF0A40E06010B6F0BEC0CF052
:105BC000A60E06010B6F0BEC0CF0C80E06010B6F56
:105BD0000BEC0CF0D30E06010B6F0BEC0CF0060176
:105BE0000B6B0BEC0CF0400E06010B6F0BEC0CF08A
:105BF000D50E06010B6F0BEC0CF0800E06010B6F3F
:105C00000BEC0CF0A80E06010B6F0BEC0CF03F0E2A
:105C100006010B6F0BEC0CF0D60E06010B6F0BECB4
:105C20000CF0800E06010B6F0BEC0CF0D90E060188
:105C30000B6F0BEC0CF0220E06010B6F0BEC0CF053
:105C4000DA0E06010B6F0BEC0CF006010B6B0BEC84
:105C50000CF0EE0E06010B6F0BEC0CF0810E060142
:105C60000B6F0BEC0CF07F0E06010B6F0BEC0CF0C6
:105C70002E0E06010B6F0BEC0CF0DB0E06010B6F0A
:105C80000BEC0CF0400E06010B6F0BEC0CF08D0EC4
:105C900006010B6F0BEC0CF0140E06010B6F0BECF6
:0E5CA0000CF0AF0E06010B6F0BEC0CF01200B7
:105CAE000501C86BC96BC7C501F00132019E0132F7
:105CBE00019E0132019E000EC95D02E10150C85DD8
:105CCE0063E2CA6BCB6B000ECB5D02E1C651CA5DBF
:105CDE0058E2CC6B080ECC5D51E2C8C500F0C9C5C8
:105CEE0001F0C6C504F0000E056E25EC03F0CA5196
:105CFE000026CB5101220050C325F66E0150C4215F
:105D0E00F76E000EC521F86E0900F5CF03F0CCC575
:105D1E0002F0010E006E000E016E025005E000361C
:105D2E0000900136FF0FFAD703500016000E011631
:105D3E000050011004E0010E00019F6F02D000011F
:105D4E009F6B0501CA51C1250601396F030E016E05
:105D5E00C8C500F0015004E000360090FF0FFBD7DD
:105D6E0000500501C22506013A6F0501CC5106010E
:105D7E003A271BEC00F00501CC2BACD7CA4BCB2B32
:0A5D8E00A2D7C84BC92B8FD7120013
:105D9800210E06011E6FFBEC06F006011E6BFBECE4
:105DA80006F07F0E06011E6FFBEC06F0220E0601C0
:105DB8001E6FFBEC06F006011E6BFBEC06F0080EEE
:105DC80006011E6FFBEC06F0D30E06011E6FFBECFE
:105DD80006F0400E06011E6FFBEC06F006010B6B89
:105DE8000C6B45EC13F00501C16B080EC15D26E292
:105DF800C151B00F06011E6FFBEC06F006011E6BC9
:105E0800FBEC06F0100E06011E6FFBEC06F0350EDB
:105E18000D6E0D2EFED70501C26B800EC25D0CE221
:105E280006010B6B7EEC13F06A0E0D6E0D2EFED77D
:105E380000000501C22BF1D7C12BD7D72E0E0601C2
:105E48001E6FFBEC06F006010B6B0C6B45EC13F0B8
:025E5800120036
:105E5A00010E00019F6F200E0501C16F000EC26F77
:105E6A00800E006E800EC219005C02E1C15100086A
:105E7A003CE2400ED16F000ED26FC1512008D36FA1
:105E8A00C2C5D4F5000ED457C1514008D56FC2C55A
:105E9A00D6F5000ED657200EC125D76F000EC221A7
:105EAA00D86F400EC125D96F000EC221DA6F200EBD
:105EBA00C125DB6F000EC221DC6F46EC25F0000124
:105ECA009F5302E09F6B02D0010E9F6F09DC150EF3
:105EDA000C6EC60E0D6E0D2EFED70C2EFCD70000D2
:105EEA00050EC15F000EC25BBBD7010E00019F6F9A
:025EFA00120094
:105EFC00010E00019F6F400E0501C16FC1510408D6
:105F0C0028E2400ED16F000ED26F200ED36F000E20
:105F1C00D46FC1C5D5F5000ED66F48EC28F075ECE2
:105F2C002BF000019F5302E09F6B02D0010E9F6F7C
:105F3C00020E0B6EA00E0C6E920E0D6E0D2EFED779
:105F4C000C2EFCD70B2EFAD70000040E0501C15FF6
:045F5C00D5D7120083
:105F60000900F5CFE6FF0006FBE10106F9E11200AA
:105F70000501C16B400EC15D1CE2400ED16F000EE9
:105F8000D26F200ED36F000ED46FC1C5D5F5000EB1
:105F9000D66F6DEC27F075EC2BF0150E0C6EC60E5F
:105FA0000D6E0D2EFED70C2EFCD70000040EC1275F
:045FB000E1D7120023
:105FB400C1C50BF6C2C50CF6C3C50DF60EEC13F045
:105FC400C1C50BF60501C451C22506010C6F0C07AF
:105FD400C3C50DF60EEC13F0C1C51EF6C2C51FF6FF
:105FE400C4C520F69AEC06F00501C351C12506018B
:105FF4001E6F1E07C2C51FF6C4C520F69AEC06F034
:02600400120088
:10600600010E00019F6F0501C16B200EC15D27E2E5
:10601600C1C50BF6C1C50CF6C1C500F0003600902F
:106026000050800806010D6F005040080E6F28ECE6
:1060360013F075EC2BF0150E0C6EC60E0D6E0D2EB4
:10604600FED70C2EFCD7000000019F5302E09F6B89
:1060560002D0010E9F6F030E0501C127D6D7010E90
:0660660000019F6F120013
:10606C00010E00019F6F0501C16B800E006E800E4A
:10607C00000A005C02E11E0EC15D29E2C1C5D1F52A
:10608C00C1C5D2F5C1C500F00036009000508008A3
:10609C00D36F00504008D46FC1C500F00032009E91
:1060AC0000501008D56F69EC28F075EC2BF0090E38
:1060BC000B6E1E0E0C6EE40E0D6E0D2EFED70C2EFE
:1060CC00FCD70B2EFAD70000040EC127CED7120036
:1060DC000501C16B200EC15D21E2400ED16FC15193
:1060EC002008D26FC1514008D36FC151200FD46F1B
:1060FC00C151400FD56FC151200FD66F0EEC25F05A
:10610C0075EC2BF0150E0C6EC60E0D6E0D2EFED70B
:0E611C000C2EFCD70000050EC127DCD71200A8
:10612A000D0E06013B6F0EEC00F00A0E06013B6FE6
:06613A000EEC00F0120063
:10614000C1C55CF5C2C55DF5C3C55EF5C4C55FF5E7
:10615000C5C5B8F5C6C5B9F5C7C5BAF5C8C5BBF557
:10616000C9C562F5CAC563F5CBC564F5CCC565F58F
:10617000CDC5BDF5CEC5BEF5CFC5BFF5D0C5C0F503
:0261800012000B
:106182001C0E0501B86F000EB96F3B0EBA6F060EFA
:10619200BB6FFF0E5C6FFF0E5D6F000E5E6F000E39
:1061A2005F6FFF0E626FFF0E636F000E646F000E73
:1061B200656FFF0EBD6FFF0EBE6F000EBF6F000E4C
:1061C200C06FAC8A900EAB6E948E949C9EAA03D044
:0861D200AECF00F0FBD7120074
:1061DA00010E00019F6F0501C16BC26B000EC25D0B
:1061EA0002E11E0EC15D35E2C1C5D1F5C1C5D2F5C8
:1061FA00C1C500F00036009000508008D36F0050EF
:10620A004008D46FC1C500F0C2C501F001320032A6
:10621A00019E00501008D56F97EC24F000019F539F
:10622A0002E09F6B02D0010E9F6F75EC2BF0090EF6
:10623A000B6E1E0E0C6EE40E0D6E0D2EFED70C2E7E
:10624A00FCD70B2EFAD70000020EC127000EC2237C
:0A625A00C5D7010E00019F6F12006E
:1062640057EC46F09B6A700ED36E9B8CD3B401D06E
:10627400FDD7290E0B6E960E0C6E7F0E0D6E0D2E35
:10628400FED70C2EFCD70B2EFAD7020E0F01386F57
:10629400396B3A6B830E926E609C929689969298B3
:1062A4008998FF0E936E9382FF0E946E948201017F
:1062B400326B336B800E3319006E800E005C02E18A
:1062C4000A0E325D11E28978150E0B6E4B0E0C6EC0
:1062D400BE0E0D6E0D2EFED70C2EFCD70B2EFAD74C
:1062E4000000324B332BE6D7346B356B306B316B9C
:1062F400296B2A6B0001A76BA86BA7C02BF1A8C060
:106304002CF10101326B336B800E3319006E800E59
:10631400005C02E1800E325D0AE2A90E3225E16ED4
:10632400000E3321E26EE66A324B332BEDD7A90E11
:106334000501666F000E676FB886030EB06E400EDF
:10634400AF6EAC841CDFFF0EC16FFF0EC26F000E78
:10635400C36F000EC46F1C0EC56F000EC66F3B0EDC
:10636400C76F060EC86FFF0EC96FFF0ECA6F000E0F
:10637400CB6F000ECC6FFF0ECD6FFF0ECE6F000EF5
:10638400CF6F000ED06FDADE110E0B6E3C0E0C6E6A
:10639400CB0E0D6E0D2EFED70C2EFCD70B2EFAD77E
:1063A4000C0E06013B6F0EEC00F0BDDE8C0E0501F9
:1063B400D16F8B0ED26F000ED36FEEEC13F0B60ECE
:1063C4000501D16F880ED26F000ED36FEEEC13F07F
:1063D400280E0501D16F870ED26F000ED36FEEEC3D
:1063E40013F0EA0E0501D16F860ED26F000ED36F43
:1063F400EEEC13F0A90E0501D16F860ED26F000EDC
:10640400D36FEEEC13F0720E0501D16F850ED26FCF
:10641400000ED36FEEEC13F0660E0501D16F860EFD
:10642400D26F000ED36FEEEC13F0B30E0501D16FF3
:106434008A0ED26F000ED36FEEEC13F01F0E05011F
:10644400D16F860ED26F000ED36FEEEC13F06BDEBD
:1064540089880AEC0AF0080E0501D16F890ED26F03
:10646400000ED36FEEEC13F0A00EC86EC7EC2BF049
:106474002F6B82B24CD0F20E0501D16F890ED26F10
:10648400000ED36FEEEC13F00501606B616B400EF0
:106494000101326F000E336F800E3319006E800ECF
:1064A400005C02E1FE0E325D13E232C1C1F53CEC48
:1064B4002CF000C02FF101012F51000803E2050167
:1064C400604B612B020E01013227000E3323E4D707
:1064D4002ADE000E0501611902E1000E601915E1C2
:1064E400620ED16F880ED26F000ED36FEEEC13F0F4
:1064F400F40E0B6E820E0C6E050E0D6E0D2EFED775
:106504000C2EFCD70B2EFAD7FF00899809D0A60EC3
:106514000501D16F890ED26F000ED36FEEEC13F02C
:10652400550E0501D16F8A0ED26F000ED36FEEECBB
:1065340013F0780E01012D6F020E2E6F80EC2DF0FA
:1065440029DCD20E0501D16F8A0ED26F000ED36FF3
:10655400EEEC13F00501C16BC26BBC0EC36F720E7F
:10656400C46F000EC56F800EC66F400EC76F57EC28
:106574002EF075EC2BF00AEC0AF0010EC16FDBEC87
:106584002CF00AEC0AF00501C16BDBEC2CF00AECF0
:106594000AF0330E0501D16F880ED26F000ED36F4F
:1065A400EEEC13F043EC29F00501C16BC26BE40E71
:1065B400C36F7C0EC46F000EC56F7F0EC66F200EB6
:1065C400C76F57EC2EF070EC2BF043EC29F005016B
:1065D400C16BC26BE40EC36F800EC46F000EC56F37
:1065E400800EC66F200EC76F57EC2EF075EC2BF0A3
:1065F40070EC2BF0DF0ED16F880ED26F000ED36FCC
:10660400EEEC13F043EC29F00501C16BC26BE40E10
:10661400C36F820EC46F000EC56F7F0EC66F200E4F
:10662400C76F57EC2EF070EC2BF043EC29F005010A
:10663400C16BC26BE40EC36F7E0EC46F000EC56FD8
:106644007F0EC66F200EC76F57EC2EF075EC2BF043
:1066540070EC2BF0750ED16F8A0ED26F000ED36FD3
:10666400EEEC13F043EC29F00501C16BC26BBC0ED8
:10667400C36F760EC46F000EC56F7F0EC66F3F0EDC
:10668400C76F57EC2EF075EC2BF070EC2BF0A40ECA
:10669400D16F8B0ED26F000ED36FEEEC13F00501A9
:1066A400C16B200EC26F03EC2CF070EC2BF07F0E4C
:1066B4000501D16F890ED26F000ED36FEEEC13F08B
:1066C40043EC29F075EC2BF0010E00019F6F0101E2
:1066D400546B556B566B576B326B336B800E33199F
:1066E400006E800E005C02E1800E325D42E21A0E02
:1066F4003225D96E000E3321DA6EDE503F080501D3
:10670400606F616B000E615B000E0101331902E1E1
:10671400000E321907E132C139F660C53AF61BECB6
:1067240000F012D054C121F655C122F656C123F609
:1067340057C124F632C125F633C126F660C527F6C3
:1067440061C528F6CAEC01F032C154F133C155F1E8
:1067540060C556F161C557F1030E0C6E120E0D6E35
:106764000D2EFED70C2EFCD700000101324B332B2B
:10677400B5D775EC2BF070EC2BF0140ED16F8A0E9C
:10678400D26F000ED36FEEEC13F00501C16B400E17
:10679400C26F03EC2CF070EC2BF0C5DC43EC29F059
:1067A400010E00019F6F740E0501D16F8B0ED26F25
:1067B400000ED36FEEEC13F0010E06010B6F020E08
:1067C4000C6F640E0D6F0EEC13F00A0E0B6F060EB9
:1067D4000C6F460E0D6F0EEC13F0140E0B6F0A0EB9
:1067E4000C6F3C0E0D6F0EEC13F01E0E0B6F100EA3
:1067F4000C6F320E0D6F0EEC13F0280E0B6F140E8F
:106804000C6F280E0D6F0EEC13F0320E0B6F180E7A
:106814000C6F1E0E0D6F0EEC13F03C0E0B6F1E0E64
:106824000C6F140E0D6F0EEC13F075EC2BF070EC76
:106834002BF00AEC0AF043EC29F0010E00019F6FE3
:10684400310E0501D16F8C0ED26F000ED36FEEECBA
:1068540013F0680E0501D16F050ED26F840ED36F4D
:106864008C0ED46F000ED56F32EC24F0140E05019B
:10687400D16F030ED26F680ED36F050ED46F010E65
:10688400D56FE4EC29F00101326B336B800E3319C0
:10689400006E800E005C02E1200E325D46E232C1E1
:1068A40004F033C105F00436049005360450800822
:1068B400006E05C001F0000E0156010E005C026E70
:1068C400000E0158036E02C052F103C053F104508C
:1068D4004008006E05C001F0000E0156010E005E76
:1068E400000E015A00C060F501C061F532C1C1F566
:1068F40032C1C2F502C0C3F500C0C4F5DAEC2FF012
:1069040075EC2BF0090E0B6E1E0E0C6EE40E0D6E64
:106914000D2EFED70C2EFCD70B2EFAD70000040E3A
:1069240001013227000E3323B1D770EC2BF043EC76
:1069340029F0940E0501D16F8A0ED26F000ED36F29
:10694400EEEC13F003EC30F075EC2BF070EC2BF064
:1069540043EC29F0260E0501D16F8B0ED26F000E89
:10696400D36FEEEC13F0B8EC2FF075EC2BF070EC69
:106974002BF043EC29F0EF0E0501D16F8A0ED26F94
:10698400000ED36FEEEC13F07EEC2FF075EC2BF0D1
:1069940070EC2BF043EC29F0580E0501D16F890EF1
:1069A400D26F000ED36FEEEC13F043EC29F036EC0B
:1069B40030F075EC2BF070EC2BF08D0ED16F880E4F
:1069C400D26F000ED36FEEEC13F043EC29F003DC2E
:1069D40075EC2BF070EC2BF043EC29F0D00E050194
:1069E400D16F8B0ED26F000ED36FEEEC13F06EEC02
:1069F40030F075EC2BF070EC2BF043EC29F0BB0E6F
:106A04000501D16F8B0ED26F000ED36FEEEC13F035
:106A14002DEC2FF075EC2BF070EC2BF043EC29F0FF
:106A2400440E0501D16F8C0ED26F000ED36FEEECC5
:106A340013F08FEC2CF075EC2BF070EC2BF0D00EE7
:106A4400D16F850ED26F000ED36FEEEC13F0640E8F
:106A54000501D16F870ED26F000ED36FEEEC13F0E9
:106A640043EC29F075EC2BF0010E00019F6F680ECA
:106A74000501D16F050ED26FE40ED36F8B0ED46F68
:106A8400000ED56F32EC24F00501D16BD26B680E89
:106A9400D36F050ED46F010ED56FE4EC29F00AEC28
:106AA4000AF0680ED16F050ED26F1E0ED36F8C0ED6
:106AB400D46F000ED56F32EC24F00501D16B010EBA
:106AC400D26F680ED36F050ED46F010ED56FE4EC50
:106AD40029F00AEC0AF0680ED16F050ED26F0B0E86
:106AE400D36F8C0ED46F000ED56F32EC24F00501F9
:106AF400D16B020ED26F680ED36F050ED46F010EE8
:106B0400D56FE4EC29F00AEC0AF0680ED16F050E9B
:106B1400D26FF80ED36F8B0ED46F000ED56F32EC9C
:106B240024F00501D16B030ED26F680ED36F050EEE
:106B3400D46F010ED56FE4EC29F070EC2BF043EC2C
:106B440029F075EC2BF00B0ED16F8B0ED26F000E6B
:106B5400D36FEEEC13F0680E0501D16F050ED26F02
:106B64008F0ED36F8C0ED46F000ED56F32EC24F0E1
:106B74000501D16BD26B680ED36F050ED46F020E74
:106B8400D56FE4EC29F0410ED16F8B0ED26F000E5D
:106B9400D36FEEEC13F0680E0501D16F050ED26FC2
:106BA400980ED36F8C0ED46F000ED56F32EC24F098
:106BB4000501D16B020ED26F680ED36F050ED46F30
:106BC400020ED56FE4EC29F070EC2BF095EC30F06C
:106BD400CD0E0501D16F890ED26F000ED36FEEEC8E
:106BE40013F043EC29F075EC2BF0010E00019F6FBC
:106BF400A90E0501666F000E676FD80E586F0F0E51
:106C0400596F490E5A6F800E5B6FA90E666F000EA6
:106C1400676F66C5C1F567C5C2F5A80EC36F8C0E54
:106C2400C46F000EC56FD80EC66F0F0EC76F490E26
:106C3400C86F800EC96F5BEC2DF066C5D1F567C5D2
:106C4400D2F5D3EC13F095EC30F00501D16BD26B97
:106C540066C5D3F567C5D4F5020ED56FE4EC29F00B
:106C6400A10E00019B6F860E9C6F020E9D6F000E9D
:106C74009E6FA90E0501666F000E676FA10EC16FAE
:106C8400860EC26F020EC36F000EC46F680EC56F0E
:106C9400050EC66FEAEC2CF0680ED16F050ED26FAC
:106CA400D3EC13F095EC30F00501D16B020ED26FEA
:106CB400680ED36F050ED46F020ED56FE4EC29F085
:086CC40070EC2BF0FF00FFD77C
:108CAE0010EE15F0920E006E010E016EE00EF66ED5
:0E8CBE00840EF76E000EF86EB0EC2FF0120070
:106CCC0000000000000000000000000000000000B8
:106CDC00000000F80000000000000033300000004D
:106CEC0000100C06100C0600000000000000000054
:106CFC0040C07840C0784000043F04043F040400C6
:106D0C00007088FC08300000001820FF211E0000D5
:106D1C00F008F000E018000000211C031E211E00EA
:106D2C0000F00888700000001E2123241927211070
:106D3C0010160E0000000000000000000000000013
:106D4C00000000E0180402000000000718204000BA
:106D5C0000020418E00000000040201807000000AA
:106D6C00404080F0804040000202010F010202000E
:106D7C00000000F0000000000101011F01010100F2
:106D8C00000000000000000080B070000000000057
:106D9C0000000000000000000001010101010101E0
:106DAC000000000000000000003030000000000077
:106DBC00000000008060180400601806010000004C
:106DCC0000E010080810E000000F102020100F0049
:106DDC00001010F8000000000020203F20200000D0
:106DEC000070080808887000003028242221300028
:106DFC0000300888884830000018202020110E0030
:106E0C000000C02010F8000000070424243F2400D8
:106E1C0000F80888880808000019212020110E00AD
:106E2C0000E0108888180000000F112020110E00BF
:106E3C0000380808C83808000000003F00000000B7
:106E4C000070880808887000001C222121221C0078
:106E5C0000E010080810E0000000312222110F00A1
:106E6C00000000C0C0000000000000303000000036
:106E7C0000000080000000000000806000000000A6
:106E8C0000008040201008000001020408102000BF
:106E9C00404040404040400004040404040404000A
:106EAC00000810204080000000201008040201009F
:106EBC00007048080808F00000000030360100009F
:106ECC00C030C828E810E0000718272423140B0052
:106EDC000000C038E0000000203C230202273820CC
:106EEC0008F8888888700000203F202020110E00B0
:106EFC00C0300808080838000718202020100800A7
:106F0C0008F808080810E000203F202020100F008F
:106F1C0008F88888E8081000203F2020232018005B
:106F2C0008F88888E8081000203F200003000000C3
:106F3C00C03008080838000007182020221E020064
:106F4C0008F808000008F808203F210101213F2023
:106F5C00000808F8080800000020203F202000004E
:106F6C0000000808F8080800C08080807F0000003E
:106F7C0008F888C028180800203F20012638200077
:106F8C0008F8080000000000203F202020203000DE
:106F9C0008F8F800F8F80800203F003F003F2000F8
:106FAC0008F830C00008F808203F200007183F0000
:106FBC00E01008080810E0000F10202020100F002F
:106FCC0008F808080808F000203F21010101000022
:106FDC00E01008080810E0000F18242438504F0067
:106FEC0008F8888888887000203F2000030C302027
:106FFC0000708808080838000038202121221C0065
:10700C00180808F8080818000000203F20000000AD
:10701C0008F808000008F808001F202020201F0096
:10702C000878880000C83808000007380E010000F6
:10703C00F80800F80008F800033C0700073C0300C0
:10704C00081868808068180820302C03032C302026
:10705C000838C800C83808000000203F2000000095
:10706C0010080808C83808002038262120201800ED
:10707C00000000FE020202000000007F40404000C1
:10708C00000C30C000000000000000010638C000F9
:10709C0000020202FE000000004040407F000000A1
:1070AC0000000402020204000000000000000000C6
:1070BC0000000000000000008080808080808080C4
:1070CC0000020204000000000000000000000000AC
:1070DC0000008080808000000019242222223F20A2
:1070EC0008F8008080000000003F112020110E00E5
:1070FC000000008080800000000E11202020110074
:10710C00000000808088F800000E112020103F2025
:10711C000000808080800000001F222222221300A9
:10712C00008080F0888888180020203F20200000F4
:10713C000000808080808000006B949494936000A9
:10714C0008F8008080800000203F210000203F20B4
:10715C0000809898000000000020203F20200000B4
:10716C00000000809898000000C08080807F0000A4
:10717C0008F8000080808000203F24022D30200081
:10718C00000808F8000000000020203F202000002C
:10719C008080808080808000203F20003F20003F46
:1071AC008080008080800000203F210000203F2054
:1071BC000000808080800000001F202020201F0005
:1071CC00808000808000000080FFA12020110E0034
:1071DC000000008080808000000E112020A0FF8025
:1071EC00808080008080800020203F2120000100D2
:1071FC000000808080808000003324242424190027
:10720C00008080E0808000000000001F2020000033
:10721C008080000000808000001F202020103F2074
:10722C00808080000080808000010E300806010004
:10723C0080800080008080800F300C030C300F00A9
:10724C0000808000808080000020312E0E312000D4
:10725C00808080000080808080818E701806010004
:10726C0000808080808080000021302C2221300022
:10727C0000000000807C020200000000003F404043
:10728C0000000000FF00000000000000FF000000F4
:10729C000002027C800000000040403F0000000023
:1072AC0000060101020204040000000000000000BE
:1072BC0000000000000000000000000000000000C2
:1072CC0000000000000000000000000000000000B2
:1072DC0000000000000000000000000000000000A2
:1072EC000000000000000000000000000000000092
:1072FC000000000000000000000000000000000082
:10730C0000000000000000000000000000800000F1
:10731C000000000000000000000000000000000061
:10732C000000000000000000000000000000000051
:10733C000000000000000000000000000000000041
:10734C000000000000000000000000000000000031
:10735C000000000000000000000000000000000021
:10736C000000000000000000000000000000000011
:10737C00000000000000000000008080E0F0F0F051
:10738C00F0F8F8FCFFFF7F7E7E3E3E1E1F1F9F9F86
:10739C001F1F1E0E3E7EFEDC84000000000000005D
:1073AC0000000000000000000000000000000000D1
:1073BC0000000000000000000000000000000000C1
:1073CC0000008080E0F0F8F8FCFEFEFEFF7F7F3FBF
:1073DC003F3F9EFEFEFC3C1C0E0E070707070703F3
:1073EC000707060E060E0E0E0C1C1C1C183818383F
:1073FC0038183818181C1C0C0E0E0F0F0F0F1F3FCF
:10740C00FFE7C301000080C0F0F81CEEF07E3F7F68
:10741C007170E0E0C00707077FE00000000000008B
:10742C000000000000000000000000000000000050
:10743C00000000000000000000080C080C1C0C1CD4
:10744C001C1E1F3F3F3F3F1F1F0F07010080800086
:10745C000080FFFFFF0E000000000000000080C055
:10746C00E0F0F0F8FCFC80000000000000000000E0
:10747C000000000000000000E0F0F8000000000038
:10748C000033FFFFFCFAF3FF7F1E0F070100000023
:10749C00000000010F0F0E1E0F0F03000000000074
:1074AC0000000000000000000000000000000000D0
:1074BC0000000000000000000000000000008080C0
:1074CC00C080800080C0C0C0C0F0F8FEEF77373FAE
:1074DC003F1BFBF9F0F0F0B0383818381C0E0F07D2
:1074EC000301010103030307070E0E0E0C1C1C38CD
:1074FC003818F8F0F0F0F0F0F3FF777F7E7CF8E0CE
:10750C00807EFFBF070703010000000000000000A1
:10751C00000000000000000000000000000000005F
:10752C00000000000000000000000000000000004F
:10753C00000000000000000000000000020F0F1F00
:10754C000F1F070F0F0F0D1F0F070360F0F0F8F858
:10755C00F0FCFEFF7F3F390000000000000000003F
:10756C000000000000000080808080C0E0F0FCFE85
:10757C00FE677F3F0F0703010000000000000F3F74
:10758C007FFFE3FFFC78000000000000000000001B
:10759C0000000000000000000000000000000000DF
:1075AC0000000000000000000000000000000000CF
:1075BC0000000000000000000000000000000000BF
:1075CC0000000000000000000000000000000101AD
:1075DC00000100000000000000000000000000009E
:1075EC0030F87C7E3E3E3F0F1F0F0F070303010058
:1075FC00000000000000000000000000000000007F
:10760C000000237FFFFFFEF8E08000000000000078
:10761C00000000000000000000000000000000005E
:10762C00000000000000000000000000000000004E
:10763C00000000000000000000000000000000003E
:10764C00000000000000000000000000000000002E
:10765C00000000000000000000000000000000001E
:10766C00000000000000000000000000000000000E
:10767C0000000000000000000000000000000000FE
:10768C00000000000001071F1F0F1F1E0400000058
:10769C0000000000000000000000000000000000DE
:1076AC0000000000000000000000000000000000CE
:1076BC0000000000000000000000000000000000BE
:1076CC0000000000000000000000000000000000AE
:1076DC00000000000000000000008080800080C0DE
:1076EC0060B0183C20B0D0C89CD4D870F0F0C0C0AA
:1076FC00C0C0C0808000000000000000000000003E
:10770C000000E0E0E0E0C08080000000000000002D
:10771C000000000000000080C04060F0F8E8EC645D
:10772C00646C7C784898F0F0E0C000000000000029
:10773C00000000000000000000000000000000003D
:10774C00000000000080602040C08080404040C0AD
:10775C004040404040607048466321B137C38104CB
:10776C000607060607050D09193323460E0C1831BA
:10777C0061830307870F1F3E7E6CC810302040408A
:10778C00C08081C3C34746C48D89991B1E1E3E3ED3
:10779C0036363212161F1F0C0C06030101000000B6
:1077AC0000000000000001030CA7FFFC000000001B
:1077BC0000000000000000000000000000000000BD
:1077CC000000000000C33C98D40C1838888CE428C6
:1077DC0018080C4ACEDC14E0800C1273F80F193325
:1077EC00C60000000000000000000000000000C007
:1077FC00E030000000C1E27478706083060800007D
:10780C000001010100000000000107FFFE061C7CC6
:10781C00F810902060C08080000000000000000084
:10782C000000008080C0E0F8FEFF3F0F0000000069
:10783C00000000000000000000000000000000003C
:10784C000000000018E7C187A60C3EF87DFD3D2125
:10785C00FAFA24681ECF4F0F90C8BC00837F00F843
:10786C00F0000000C0800000000F0F1EFEFFFFFFA5
:10787C00F0E0000807030080E0F81E070100E000BC
:10788C000000C08000000000000000C18F18000044
:10789C00030401070E1E3F7FBDB93B7A7E3E3E3A84
:1078AC003A3F1D1F0F0F07030100000000000000EE
:1078BC0000000000000000000000000000000000BC
:1078CC000000000000010301033FC00F3843504883
:1078DC003F0FC36018CDF5F7F7EFF7E7EFDE9F1F0B
:1078EC007FFDFCFEFFFFFF7E7C7C7E7FFFFFFF03A6
:1078FC0000010020B0FCFEFFFFE1E0F0FCFFFFF810
:10790C00FCFFFFFFFFFEFCFC78F8F8FFFFFFFCF824
:10791C00E0C0C0C4F8F0E080808191E2C2840C0821
:10792C0018102060C0800000000000000000000063
:10793C00000000000000000000000000000000003B
:10794C0000000000000000000000010382C6462673
:10795C00321B8CC6F3FDFFFFFFFFFF7F3F1F0F079E
:10796C000E18313D0909191C0E86C7F37F3F1F4CB9
:10797C00E6F2F8FEFFFF1F0307070F1F1F1F3F3F15
:10798C003F7F7F7F7F7F7FFFFFFFFEFDFDF9FB7B4E
:10799C00332303070707070F0F0F3FFFFFFFFFFE00
:1079AC00FC7800F7FF01010000000000000000005F
:1079BC00000000000000000000000000008080C0FB
:1079CC00C0C0C04040209088E4F2FBFDFCF0F8FC05
:1079DC00FEFF7F7F3F3F1F0F070301000000008069
:1079EC008080C040C0D0585CFFFFFFFFFFFFFFFF4F
:1079FC00FF7F1F0F03000000000000000080C0C0CC
:107A0C00C0C0C0C0C0E0F8FFFFFFFFFF3F07010090
:107A1C000000000000F0F838F8FCFF3F1BFBF7EB10
:107A2C002170FECF000000000000000000000000EC
:107A3C00000010101010181818181C1C1C1B181FF4
:107A4C001F1F1F1F1F1F1F1F1F1F1F1F1B1B19194E
:107A5C00181818181010101818181818181C1F1CA3
:107A6C0016181C1C111818181F1F1F1F1F1F1F1B57
:107A7C0018181810101010101818181C1E191C1F8C
:107A8C001F1F1F1F1F1F1F1F1F1F1F1C1818101029
:107A9C001018181C1C1F1F18101F1F1C181F1F1F2D
:107AAC00101F1F1B181818181010000000000000E1
:107ABC000000000000000000002F00000000070084
:107ACC00070000147F147F1400242A7F2A120062FE
:107ADC0064081323003649552250000005030000AA
:107AEC0000001C224100000041221C000014083E32
:107AFC0008140008083E0808000000A060000008F8
:107B0C00080808080000606000000020100804024B
:107B1C00003E5149453E0000427F40000042615109
:107B2C004946002141454B31001814127F100027A3
:107B3C0045454539003C4A49493000017109050366
:107B4C0000364949493600064949291E0000363697
:107B5C0000000000563600000008142241000014FA
:107B6C0014141414000041221408000201510906D7
:107B7C0000324959513E007C1211127C007F494958
:107B8C004936003E41414122007F4141221C007F89
:107B9C0049494941007F09090901003E4149497A97
:107BAC00007F0808087F0000417F41000020404111
:107BBC003F01007F08142241007F40404040007F7D
:107BCC00020C027F007F0408107F003E4141413EC1
:107BDC00007F09090906003E4151215E007F091909
:107BEC0029460046494949310001017F0101003F06
:107BFC004040403F001F2040201F003F4038403F86
:107C0C0000631408146300070870080700615149E9
:107C1C00454300007F414100000204081020000091
:107C2C0041417F00000402010204004040404040FA
:107C3C00000001020400002054545478007F484492
:107C4C00443800384444442000384444487F0038C9
:107C5C005454541800087E0901020018A4A4A47CF2
:107C6C00007F080404780000447D400000408084BC
:107C7C007D00007F102844000000417F4000007C04
:107C8C0004180478007C0804047800384444443810
:107C9C0000FC242424180018242418FC007C08045C
:107CAC00040800485454542000043F444020003C35
:107CBC004040207C001C2040201C003C4030403CBC
:107CCC00004428102844001CA0A0A07C004464544C
:087CDC004C4414141414141498
:107CE400FFFFFFFFFFFFFFFFFFFFFFFFFFFFFFFFA0
:107CF400FFFFFFFFFFFFFFFFFFFFFFFFFFFFFFFF90
:107D0400FFFFFFFFFFFFFFFFFFFFFFFFFFFFFFFF7F
:107D1400FFFFFFFFFFFFFFFFFFFFFFFFFFFFFFFF6F
:107D2400FFFFFFFFFF0703F3030303E3A3A3A3A3DF
:107D3400A3A3A3A3A3E34303038383C3C3C3E3E3CF
:107D4400E3E3E3E3E3E3E3E3E3E3E3E3E3C3C3C35F
:107D5400C38303030303030303F30307FFFFFFFFCB
:107D6400FFFFFFFFFFFFFFFFFFFFFFFFFFFFFFFF1F
:107D7400FFFFFFFFFFFFFFFFFFFFFFFFFFFFFFFF0F
:107D8400FFFFFFFFFFFFFFFFFFFFFFFFFFFFFFFFFF
:107D9400FFFFFFFFFFFFFFFFFFFFFFFFFFFFFFFFEF
:107DA400FFFFFFFFFF0000FF000000ACACECECC8DD
:107DB400C8E8E8A8000000FEFFFFFFFFFFFFFFFF89
:107DC400FFFFFFF1606060607F7F7F7F7F7F7F7F49
:107DD4007F7F7F7F7C00000000FF0000FFFFFFFF2C
:107DE400FFFFFFFFFFFFFFFFFFFFFFFFFFFFFFFF9F
:107DF400FFFFFFFFFFFFFFFFFFFFFFFFFFFFFFFF8F
:107E0400FFFFFFFFFFFFFFFFFFFFFFFFFFFFFFFF7E
:107E1400FFFFFFFFFFFFFFFFFFFFFFFFFFFFFFFF6E
:107E2400FFFFFFFFFF0000FF000000D2505052523E
:107E3400525252524000003F7FFFFFFFFFFFFFFFFF
:107E4400FFFFFFC080808080C0FEFEFEFEFEFEFEBF
:107E5400FEFE7E7E1E00000000FF0000FFFFFFFF0D
:107E6400FFFFFFFFFFFFFFFFFFFFFFFFFFFFFFFF1E
:107E7400FFFFFFFFFFFFFFFFFFFFFFFFFFFFFFFF0E
:107E8400FFFFFFFFFFFFFFFFFFFFFFFFFFFFFFFFFE
:107E9400FFFFFFFFFFFFFFFFFFFFFFFFFFFFFFFFEE
:107EA400FFFFFFFFFFF0E0E7E0E0E0E3E2E2E2E211
:107EB400E2E2E2E2E2E2E2E2E2E0E0E1E1E1E1E3A5
:107EC400E3E3E3E3E3E3E3E3E3E3E3E3E3E1E1E184
:107ED400E0E0E0E0E0E0E0E0E8E7F0F0FFFFFFFFF3
:107EE400FFFFFFFFFFFF7F7F7F7F7FFFBFBFBFBF1E
:107EF400BFBFBFBFBFBFBFBFBFBFBFBFBFBFBFBF8E
:107F0400BF3F3F3F3FBFFFBFBFBFBFFF7FFFFFFF7D
:107F1400FFFFFFFFFFFFFFFFFFFFFFFFFFFFFFFF6D
:107F2400FFFFFFFFFFFFFFFFFFFFFFFFFFFFFFFF5D
:107F3400FFFFFFFFFFFFFFFFFFFFFFFFFFFFFFFF4D
:107F4400FFFFFFFFFFFFFFFFFFFFFFFFFFFFFFFF3D
:107F5400FFFFFFFFFFFFFFFFFFFFFFFFFFFFFFFF2D
:107F6400FFFF813F3E3E00001E1E3E00003E3E00DD
:107F740000220606220000003E0000000018007ED9
:107F84007E112FCDEDEDEDEDEDEDE399BFFEFEE3BA
:107F9400F7F3DFD7B7B7FFCFBFEF1F5FBFFFFFFF19
:107FA400FFFFFFFFFFFFFFFFFFFFFFFFFFFFFFFFDD
:107FB400FFFFFFFFFFFFFFFFFFFFFFFFFFFFFFFFCD
:107FC400FFFFFFFFFFFFFFFFFFFFFFFFFFFFFFFFBD
:107FD400FFFFFFFFFFFFFFFFFFFFFFFFFFFFFFFFAD
:107FE400FFFF3F1F1F0E0E0E0E00000000003000AA
:107FF4007830220204180000000000000000000095
:10800400000001010101010101030E0F0F0F0F0315
:10801400010111597119011734352B3FF3FFFFFF8B
:10802400FFFFFFFFFFFFFFFFFFFFFFFFFFFFFFFF5C
:10803400FFFFFFFFFFFFFFFFFFFFFFFFFFFFFFFF4C
:10804400FFFFFFFFFFFFFFFFFFFFFFFFFFFFFFFF3C
:10805400FFFFFFFFFFFFFFFFFFFFFFFFFFFFFFFF2C
:10806400FFFFFEFEFEFCFCFCFCFCFCFCFCFCFCF844
:10807400F8F8F0F0F0F0F0F0E0F0F0F0F0F0E0E01C
:10808400E0E0E0E0C0C0C0C0E0A0E080A0E0E0C06C
:10809400C0C0C0C0F0F8F8F8F8F8FCFEFEFFFFFF1F
:1080A400FFFFFFFFFFFFFFFFFFFFFFFFFFFFFFFFDC
:1080B400FFFFFFFFFFFFFFFFFFFFFFFFFFFFFFFFCC
:1080C400FFFFFFFFFFFFFFFFFFFFFFFFFFFFFFFFBC
:1080D400FFFFFFFFFFFFFFFFFFFFFFFFFFFFFFFFAC
:1080E400FFFFFFFFFFFFFFFFFFFFFFFFFFFFFFFF9C
:1080F400FFFF7F1F1118C8CCCECEDF9FFFFFFFFF0D
:10810400FF7F7F7F7F7E3800000000021F1F33C780
:108114000F0F3F7FFFFFFFFFFFFFFFFFFFFFFFFF8B
:10812400FFFFFFFFFFFFFFFFFFFFFFFFFFFFFFFF5B
:10813400FFFFFFFFFFFFFFFFFFFFFFFFFFFFFFFF4B
:10814400FFFFFFFFFFFFFFFFFFFFFFFFFFFFFFFF3B
:10815400FFFFFFFFFFFFFFFFFFFFFFFFFFFFFFFF2B
:10816400FFFFFFFFFFFFFFFFFFFFFFFFFF47F3815D
:10817400C1F0F8FCFCFCFCFCBC9D9D3F1F0F037987
:10818400FDF4E6E6C68E820000000000000000F860
:10819400F8BE3E201025FFFFFFFFFFFFFFFFFFFF9C
:1081A400FFFFFFFFFFFFFFFFFFFFFFFFFFFFFFFFDB
:1081B400FFFFFFFFFFFFFFFFFFFFFFFFFFFFFFFFCB
:1081C400FFFFFFFFFFFFFFFFFFFFFFFFFFFFFFFFBB
:1081D400FFFFFFFFFFFFFFFFFFFFFFFFFFFFFFFFAB
:1081E400FFFFFFFFFFFFFFFFFFFFFFFF790E070702
:1081F400071CFFFFFF030144448409091903028794
:10820400FFF71F070301000000000040C000301703
:1082140039000080F6FFFFFFFFFFFFFFFFFFFFFFB6
:10822400FFFFFFFFFFFFFFFFFFFFFFFFFFFFFFFF5A
:10823400FFFFFFFFFFFFFFFFFFFFFFFFFFFFFFFF4A
:10824400FFFFFFFFFFFFFFFFFFFFFFFFFFFFFFFF3A
:10825400FFFFFFFFFFFFFFFFFFFFFFFFFFFFFFFF2A
:10826400FFFFFFFFFFFFFFFFFFFFFFFFC0829280C2
:108274000000C30F0F1F1E1E1E1E1C1C1C0E0F070A
:108284000B040200000000000000000000000000D9
:1082940000B8FEFFFFFFFFFFFFFFFFFFFFFFFFFF31
:1082A400FFFFFFFFFFFFFFFFFFFFFFFFFFFFFFFFDA
:1082B400FFFFFFFFFFFFFFFFFFFFFFFFFFFFFFFFCA
:1082C400FFFFFFFFFFFFFFFFFFFFFFFFFFFFFFFFBA
:1082D400FFFFFFFFFFFFFFFFFFFFFFFFFFFFFFFFAA
:1082E4000000000000F0F8F8F878787878F8F0E00A
:1082F400E08000000000000000000000000000001A
:108304000000000000000000000000000000000069
:10831400000000F0F0F8F000000000F8F8F8F87839
:10832400787878787878787070100000000000F021
:10833400F0F0F00000000000000000000000000069
:10834400000000000000000000F0F0F0F000000069
:108354000000000000000000000000000000000019
:1083640000000000FFFFFFFFF0F0F0F0F87F1F1F98
:108374000F00000080F0F8F87E1E1E1EFEF8F8F8CC
:1083840000000000F8F8F8F800000000F8F8F8F829
:108394000000FFFFFFFF00000000FFFFFFFF7878F1
:1083A4007878787878781010000000000000F8F8E9
:1083B400F8F800000000F8F8F8F800000000F8F8F9
:1083C400F8F8000000000000F8FEF8F800008080D3
:1083D400F0F87E7E1E1E7E7EFEF8E0E000000000C7
:1083E400000000FFFFFFFF0000000000000000008D
:1083F4000000001FFFFFFFE0E0E0E0FFFFFFFFE001
:108404000000007FFFFFFFE0E0E0E0FFFFFFFF0070
:1084140000FFFFFFFF00000000FFFFFFFF00000060
:10842400000000000000000000000000000707FF3B
:10843400FFF8F800007F7FFFFFE0E0E0E0FFFFFFD0
:10844400FF00000000000007FFFFFFF8001F1FFFF0
:10845400FFF0F0E0E0F0F0FF7F1F1F0000000000DD
:108464000000000100000000000000000000000007
:1084740000000000010101010101000001010100EF
:1084840000000000010101010101010101010000DE
:1084940000000100000000000000010000000000D6
:1084A400000000000000000F1F1F7EF8F0F0FF7FA7
:1084B4001F1F000000000001010101010101010171
:1084C4000F0F1F7EF8F8F0FF7F7F1F0000000000F1
:0C84D40001010101010100000000000096
:0484E0000000000098
:0184E4000097
:1084E5002024282C303336383A3B3C3C3C3C3B3A44
:1084F5003A393837373636363737383839393A3AF8
:108505003A3A3A39393838373736363637373839E7
:108515003A3A3B3C3C3C3C3B3A383633302C2824F9
:10852500201C1814100D0A08060504040404050689
:1085350006070809090A0A0A0909080807070606B5
:108545000606060707080809090A0A0A09090807A5
:10855500060605040404040506080A0D1014181C73
:018565000015
:048566000000000011
:01856A00010F
:07856B00286E756C6C2900FD
:1085720020417574726573203A204472697665727F
:108582005F4F6C65645F493243315F48575F3138F2
:108592004678784B32325F323032315F30332E6878
:1085A2002C206574204472697665725F4F6C656435
:1085B2005F493243315F48775F31384678786B32B2
:0E85C200325F323032315F30332E630D0A00EB
:1085D0000D0A206D6F64652065637269747572653C
:1085E000206469726563742064616E73204F4C452A
:1085F0004420636F6E6669672031323878363420E4
:108600002C2073616E7320706173736572207061CA
:0F86100072206C6520627566666572200D0A0027
:10861F00204861726477617265203A2043617274F9
:10862F006520426173652031384632364B32322C29
:10863F00204C4344204F4C454420302E39362220C5
:10864F00313238783634204A61756E652065742072
:07865F00426C65750D0A0075
:1086660020436F6E666967203A20503138463236AD
:108676004B32325F464F53435F696E7465726E6567
:108686005F313678504C4C5F36344D487A5F5241F4
:10869600365F467265714F75742E636667736368DD
:0386A6000D0A00BA
:1086A90020536F75726365203A20426173655F31AB
:1086B900384632364B32325F546573745F4F4C45DE
:1086C900445F4932435F31323878363420766572F7
:1086D90073696F6E20323032315F303331320D0AB7
:0186E9000090
:1086EA002050726F6A6574203A20426173655F3167
:1086FA00384632364B32325F546573745F4F4C459D
:10870A00445F493243315F48575F313238783634F3
:0E871A005F323032312E6D637070690D0A00CF
:10872800204469726563746F7279203A20433A5C19
:108738005F4D696B726F435C5F4D657350726F6A12
:108748006574735F4D696B726F435C5F424153455B
:0C8758005F31384632364B32320D0A00D9
:1087640020746578742031392063686172732073D2
:10877400697A6520312028666F6E7420367838292E
:1087840020313233343536373839303132333435B9
:07879400363738390D0A00E9
:10879B000000007F000020820000488500007A88DE
:1087AB0000401C8C0050438F0024749280961896C6
:1087BB0020BC3E99286B6E9CF90215A0EC782DC15C
:0487CB00CAF249E2C3
:1087CF000000007FCDCC4C7B0AD723786F12037546
:1087DF0017B75171ACC5276EBD37066B95BF56677E
:1087EF0077CC2B645F700961FFE65B5D08E53C3C6D
:0487FF006042221B97
:10880300010000000800000040000000000200001A
:1088130000100000008000000000040000002000A1
:1088230000000001000000080000004000000000FC
:10883300203220696D6167657320313238783332B5
:10884300203A204D6172796C696E204D6F6E726FA4
:0F88530065206574204D696B726F45200D0A001A
:10886200204E6F2064657669636520666F756E645D
:1088720020206F6E204932433120627573202121FE
:0B88820021212121212121200D0A00CD
:10888D002052656374616E676C657320506C656909
:10889D006E73206176656320636F696E73206172FC
:0988AD00726F6E6469730D0A001C
:1088B60020506F77657220737570706C793A20342A
:1088C6002E302056206D696E692021207570207427
:0988D6006F20352E30560D0A000A
:1088DF00203220696D616765732031323878333209
:1088EF00203A207061756C666A756A6F2065742016
:0988FF00547275636B200D0A0030
:1089080020496E6974204932433120486172647786
:10891800617265205243333D53434C202052433407
:088928003D534441200D0A00FB
:10893000010000000A00000064000000E8030000DD
:1089400010270000A086010040420F00809698008A
:0889500000E1F50500CA9A3BA5
:108958002052656374616E676C657320766964651F
:10896800206176656320636F696E73206172726F30
:078978006E6469730D0A0033
:10897F002044657373696E652073696E75736F69D3
:10898F0064652061766563206861726D6F6E6971D1
:07899F00756573200D0A004D
:1089A6002050617320646520726563686572636830
:1089B600657220446576696365206361722052435F
:0789C600313D31200D0A00D4
:1089CD002020546578746520616666696368616707
:1089DD00652050492020656E207461696C6C65209E
:0589ED0032200D0A001C
:1089F20020526563686572636865204F4C45442068
:108A0200737572206C652042757320493243200DC4
:028A12000A0058
:108A1400205363726F6C6C2073696E75736F696435
:108A2400652076657273206C6520686175740D0A23
:018A34000041
:108A3500010000001000000000010000001000000F
:108A450000000100000010000000000100000010FF
:108A550020496E6974204F4C4544205353443133AB
:108A65003036204C4344203132387836340D0A00F4
:108A7500203120696D616765203A20546967726508
:0F8A85005F3132387836345F626D70200D0A0031
:108A9400204D756C7469706C652072656374616EC9
:0F8AA400676C657320506C65696E73200D0A0056
:108AB30020464F534320203A2031364D487A2078C0
:0F8AC30020504C4C203D2036344D487A0D0A008F
:108AD20020696D6167653420313238783634202858
:0D8AE20043292063686576616C200D0A0051
:108AEF00204D756C7469706C6520636572636C657D
:0C8AFF007320506C65696E73200D0A0036
:108B0B0020746578742073697A652032202841427D
:0B8B1B0043444546474829200D0A004E
:108B2600204D756C7469706C657320636572636C37
:0B8B360065732056696465730D0A002A
:108B410020746578742073697A6520322028303169
:0B8B510032333435363729200D0A007E
:108B5C000D0A204465766963652061742061647236
:088B6C0065737365203A2000D7
:108B7400202064726177203520466173744C696EDD
:088B840065732048200D0A0072
:108B8C00204D4355203A2031384632364B32322074
:088B9C0044495032380D0A0073
:108BA40020696D616765207363726F6C6C20546912
:078BB400677265200D0A0045
:108BBB0020547269616E676C657320506C65696EC9
:058BCB0073200D0A00FB
:108BD00020547269616E676C657320766964657391
:048BE000200D0A005A
:108BE400313233343536373839303132333435363F
:048BF40037383900D5
:108BF8004C69676E6520342055565758595A2020BD
:038C080020200029
:108C0B004C69676E652033204B4C4D4E4F50515283
:038C1B00535400AF
:108C1E004C69676E652032204142434445464748C1
:038C2E00494A00B0
:108C310020647261772072656374616E676C65731D
:038C41000D0A0019
:108C4400205363726F6C6C696E6720746578740D61
:028C54000A0014
:108C5600303132333435363738394142434445466C
:018C6600000D
:108C6700303132333435363738396162636465669B
:018C770000FC
:0C8C780020666F756E64204F4B0D0A00E3
:0B8C840072656374616E676C657300BD
:098C8F00414243444546474800B8
:098C980030313233343536370037
:078CA1005363726F6C6C005D
:068CA80025352E356600A3
:020000040030CA
:0D000100191E3CFFAF80FF0FC00FE00F4045
:00000001FF
